:100000000C9401030C9489040C9433030C94330373
:100010000C9433240C9433030C9433030C94330367
:100020000C9433030C9433030C9433030C94330378
:100030000C9433030C9433030C9433030C94330368
:100040000C947E310C9433030C949F330C94ED3359
:100050000C9433030C9433030C9433030C94330348
:100060000C9433030C94330305A84CCDB2D44EB991
:100070003836A9020C50B9918688083CA6AAAA2A4B
:10008000BE000000803F710272027B0282028A027F
:1000900092029B02A502A902AC02B702C202CC02E4
:1000A000D402D902E102E902F20245584954005350
:1000B0004156452B45584954003C504147453E0068
:1000C000F90202030F031C03290333033C03450316
:1000D0004D03550365036E0372037F038D03A00375
:1000E000AD03BE03A003D003D603DD03EA03D603AA
:1000F000F303FB030804150422042E0441044D04F9
:10010000590461046B047A0483048E0496049D04EC
:10011000A604AC04B204B804C0044D455400494DD3
:100120005000355600312E315600CA04D804E5047B
:10013000EB04F104FA04FF040B051B051C052D0557
:100140003C051B054C05500554055E056705790502
:100150001D1A1D1C1D191D1C1D1B1D1C1D181D1CE1
:100160001D1A1D1C1D191D1C1D1B1D71028A0593C6
:10017000059D050C00003C000000018A04C8000039
:100180000000000100C8003264010101000000010C
:10019000000000010100000100000100000000005B
:1001A000010101010100010100040000000500013E
:1001B000006464641E4D574F5344002020202000EB
:1001C000000000960000000004F401580220C03432
:1001D000C036C0B7C090C054C024C072C028C0CBC5
:1001E000C0CAC060C17EC17EC137C110011D0102FD
:1001F000C00FC04DC1F3C06BC12FC171C178C1C266
:10020000C0BBC0BBC0030007007AC055C106C15CBB
:10021000C03400C30064C05301BA0018C1DCC02060
:10022000007BC12A002100900054002400720027A6
:10023000003500CB0060017EC17EC137C110011DB9
:100240000102000F004C01F2006BC12FC175017F4C
:1002500001C200BB00BB00030007007A0055010685
:10026000015C003400C50064005701BA001801DCCD
:10027000C00044495341524D4544002041524D4530
:1002800044004E4F204441544100204E4F204750DF
:1002900053004C4F572053415453004C4F57205656
:1002A0004F4C5453004F4646004F4E005354415458
:1002B0004953544943530050494420434F4E464903
:1002C000470052432054554E494E4700564F4C5418
:1002D00041474500525353490043555252454E54ED
:1002E00000444953504C415900414456414E434506
:1002F0004400414C41524D5300464C592054494D05
:100300004500544F542044495354414E4345004DF9
:1003100041582044495354414E4345004D415820D3
:10032000414C544954554445004D41582053504583
:100330004544004D41482055534544004D41582007
:10034000414D5053005243205241544500524320E6
:100350004558504F00524F4C4C2050495443482070
:100360005241544500594157205241544500545080
:1003700041005448524F54544C45204D4944005478
:1003800048524F54544C45204558504F004449530F
:10039000504C4159204D41494E20564F4C5453002A
:1003A00041444A55535420564F4C5453004D4149F3
:1003B0004E20564F4C545320414C41524D0044491D
:1003C00053504C41592056494420564F4C545300E9
:1003D00043454C4C53005553452046430044495334
:1003E000504C4159205253534900534554205253C5
:1003F0005349005553452050574D00534554205202
:10040000535349204D4158005345542052535349AA
:10041000204D494E00444953504C415920414D50C4
:100420005300444953504C4159204D4148005553C5
:1004300045205649525455414C2053454E534F5236
:100440000041444A55535420414D50530041444AC1
:10045000555354205A45524F00484F52495A4F4E17
:1004600000534944452042415253005343524F4C9C
:100470004C494E472042415253005448524F545425
:100480004C450047505320434F4F5244530053456F
:100490004E534F52530047494D42414C004D41503D
:1004A000204D4F444500554E495453005620524567
:1004B00046004445425547004D41472043414C00CA
:1004C0004F53442054582043480044495354414E0C
:1004D0004345205831303000414C5449545544452F
:1004E000205831300053504545440054494D455241
:1004F000004D4148205831303000414D5053005498
:1005000045585420414C41524D53004D574F534490
:10051000202D20312E362E352E5800004D454E55BB
:100520003A54485254204D4944444C450020202020
:10053000202B594157205249474854002020202061
:100540002B50495443482046554C4C0049443A00EE
:1005500053493A004155544F2D4E54534300415591
:10056000544F2D50414C004E4F5420444554454368
:100570005445442D4E545343004E4F54204445544B
:1005800045435445442D50414C004155544F205251
:100590005448004155544F20484F4C4400204D4989
:1005A0005353494F4E0000000000240027002A004A
:1005B00000000000250028002B00000000002300A0
:1005C00026002900040404040404040402020202B4
:1005D0000202030303030303010204081020408006
:1005E0000102040810200102040810200000000786
:1005F00000020100000304060000000000000000EB
:100600005935E5E6F7E085EA98E001C08193EF3FD0
:10061000F907E0F3D9F311241FBECFEFD8E0DEBF16
:10062000CDBF11E0A0E0B1E0E2E5F2E702C0059045
:100630000D92AA35B107D9F717E0AAE5B1E001C0DC
:100640001D92A536B107E1F716E0C2E0D6E004C07E
:100650002297FE010E942339C030D107C9F70E94BA
:1006600046330C9427390C940000FB01DC0102C0D6
:1006700005900D9241505040D8F70895FB019F011D
:10068000E8944230C4F04532B4F44A3029F497FB80
:100690001EF4909581959F4F642F77270E94B13863
:1006A000805D8A330CF0895D8193CB010097A1F7BF
:1006B00016F45DE251931082C9010C945F03DC01D2
:1006C000FC01672F71917723E1F7329704C07C9189
:1006D0006D9370836291AE17BF07C8F30895609160
:1006E0003E0370913F036115710529F080E090E0B1
:1006F0000E94DE360EC06091730370917403809186
:1007000075039091760320E030E044EB53E40E94BF
:1007100045360E94AD3630E080910A0224E6829F81
:10072000C0011124861797070CF431E0832F089538
:1007300080918901882329F080E090E1A0E0B0E079
:100740005AC080918801882329F08FE996E0AEE2B3
:10075000B0E051C08AE090E0A2E0B0E08093C30531
:100760009093C405A093C505B093C60520911203CC
:1007700021FF0CC08AE190E0A2E0B0E08093C305C5
:100780009093C405A093C505B093C60580917601EA
:10079000813089F08091C3059091C405A091C50571
:1007A000B091C60581608093C3059093C405A09362
:1007B000C505B093C60523FF11C08091C305909174
:1007C000C405A091C505B091C605806A8093C30594
:1007D0009093C405A093C505B093C6058091D1013F
:1007E000882389F48091C3059091C405A091C50523
:1007F000B091C60598608093C3059093C405A093FB
:10080000C505B093C60580910102882321F480912B
:10081000FB01882389F08091C3059091C405A091C4
:10082000C505B091C60591608093C3059093C4053A
:10083000A093C505B093C6058091C7059091C805E2
:10084000A091C905B091CA052091C3053091C40596
:100850004091C5055091C60582239323A423B52357
:100860008093C7059093C805A093C905B093CA05A6
:100870000895809124038823C9F180911C03882363
:10088000A9F160913503709136036115710571F11D
:10089000809113029B0140E050E0882349F0CA0197
:1008A000B9010E94DE3621EB32E047E55BE308C088
:1008B000CA01B9010E94DE362FE632E143E85AE36D
:1008C0000E94D6379B01AC016091AD067091AE06D7
:1008D0008091AF069091B0060E94DA356093AD0624
:1008E0007093AE068093AF069093B0066091AD060C
:1008F0007091AE068091AF069091B0060E94B2361C
:1009000060938D0370938E0380938F039093900375
:1009100008951F920F920FB60F9211241092D605D0
:100920000F900FBE0F901F901895982F5E982091F2
:100930001402222311F480E001C080E41EBC0DB437
:1009400007FEFDCF3EB58EBD0DB407FEFDCF8EB5C3
:1009500089E08EBD0DB407FEFDCF8EB59EBD0DB4F2
:1009600007FEFDCF8EB5EAE8F1E080E04AE03BE02B
:100970004EBD0DB407FEFDCF9EB58EBD0DB407FE76
:10098000FDCF9EB590813EBD0DB407FEFDCF5EB597
:100990009EBD0DB407FEFDCF9EB58F5F31968633A9
:1009A00039F788E08EBD0DB407FEFDCF8EB580EA25
:1009B0008EBD0DB407FEFDCF8EB580EA8EBD0DB4A1
:1009C00007FEFDCF0EB405FCF9CF222311F48CE015
:1009D00001C08CE41EBC0DB407FEFDCF9EB58EBDDC
:1009E0000DB407FEFDCF8EB55E9A0895DF92EF92AB
:1009F000FF920F931F93CF93DF93EC018B01F22EA5
:100A000097FD02C0EE2405C0D095C195DF4FEE24BE
:100A1000E394F801E40FF11D10822EE2D22E4F155F
:100A200031F44150F801E40FF11DD082FF24415010
:100A3000F801E40FF11DCE016AE070E00E94C538B4
:100A4000805D8083442359F0CE016AE070E00E940B
:100A5000C538EB01FF2019F76115710501F7EE208C
:100A600079F0442369F04150F801E40FF11D8DE263
:100A7000808306C04150F801E40FF11D808301C05E
:100A800080E24423B9F7C801DF91CF911F910F9104
:100A9000FF90EF90DF9008958F929F92AF92BF9258
:100AA000CF92DF92EF92FF920F931F93CF93DF933A
:100AB0005A01922E97FF08C0909580957095619588
:100AC0007F4F8F4F9F4F0E2D26E0920E24E630E091
:100AD00040E050E00E94FA38C901DA016C017D0162
:100AE000F501E90DF11D8AEF980E1082192D1B5F9B
:100AF000F501E10FF11D00834EE2842E812F81501C
:100B0000191531F4182FF501E80FF11D8082F6CF89
:100B1000182FE501C80FD11DC701B6012AE030E04A
:100B200040E050E00E94FA38605D68831123D1F004
:100B3000C701B6012AE030E040E050E00E94FA38F8
:100B4000C901DA016C017D011330C0F6C114D10472
:100B5000E104F10499F606C01150F501E10FF11D11
:100B6000808301C080E21123B9F7C501DF91CF91E5
:100B70001F910F91FF90EF90DF90CF90BF90AF90BB
:100B80009F908F9008954F925F926F927F928F9275
:100B90009F92AF92BF92CF92DF92EF92FF920F930C
:100BA0001F93CF93DF937B018C015A01522E222396
:100BB00019F078E0D72E02C065E0D62EF501ED0DD4
:100BC000F11D1082DA946D2C772467FC70946A0C06
:100BD0007B1CDA948D2C992487FC90948A0C9B1CA6
:100BE000DA94CD2DDD27C7FDD09583E0D80ECA0D50
:100BF000DB1DC52C5AE3452EC801B7012AE030E0C1
:100C000040E050E00E94D838605DF3016083C80185
:100C1000B7012AE030E040E050E00E94D838122FBF
:100C2000032FF42EE52E622F732F842F952F26E0AD
:100C300030E040E050E00E94D838605DF40160830D
:100C4000612F702F8F2D9E2D26E030E040E050E088
:100C50000E94D838C901DA017C018D014882CA940A
:100C60008DEF9FEF680E791E880E991E23979FEFD8
:100C7000C91611F6852D880F850DD81AEDEFDE0EF9
:100C8000DA94CD2DDD27C7FDD095D394CA0DDB1D99
:100C9000DA94C801B7012AE030E040E050E00E9459
:100CA000D838605D6883C801B7012AE030E040E0D1
:100CB00050E00E94D838C901DA017C018D01E114AD
:100CC000F1040105110551F4DA94ED2DFF27E7FD3C
:100CD000F095D394EA0DFB1D80E207C02197DD203B
:100CE000B9F605C0DA9480833197DD20D9F7C501C4
:100CF000DF91CF911F910F91FF90EF90DF90CF90F8
:100D0000BF90AF909F908F907F906F905F904F902B
:100D1000089580916A01882309F4B6C120911403D3
:100D20003091150340911603509117038091D6011D
:100D30009091D701A0E0B0E082239323A423B523B0
:100D40000097A105B10511F1809124028823F1F0EB
:100D50001092B10586E18093AF0587E18093B005DD
:100D600060918C0270918D02CB018070907C8050DC
:100D7000904C61F4DB01B170A153BC4FEFEAF5E098
:100D800002C08D93319680818823D9F780912A0201
:100D9000882309F463C08091D20190E0A0E0B0E024
:100DA00082239323A423B5230097A105B10579F4E9
:100DB0008091D30190E0A0E0B0E082239323A423AC
:100DC000B5230097A105B10511F460E004C080EAE5
:100DD0008093AF0561E08091D40190E0A0E0B0E0A5
:100DE00082239323A423B5230097A105B10539F0ED
:100DF000E62FF0E0E155FA4F82EA80836F5F809141
:100E0000D50190E0A0E0B0E082239323A423B52392
:100E10000097A105B10539F0E62FF0E0E155FA4F52
:100E200081EA80836F5FE62FF0E0E155FA4F108290
:100E300060915C0270915D02CB018070907C80506B
:100E4000904C61F4DB01B170A153BC4FEFEAF5E0C7
:100E500002C08D93319680818823D9F78091DC017F
:100E60009091DD01A0E0B0E082239323A423B52379
:100E70000097A105B10539F01092B1058AEA809377
:100E8000AF058BEA6DC08091D8019091D901A0E0A7
:100E9000B0E082239323A423B5230097A105B105D5
:100EA00049F08DE98093AF058EE98093B0051092EB
:100EB000B10558C08091DA019091DB01A0E0B0E06B
:100EC00082239323A423B5230097A105B10539F00C
:100ED0001092B1058DEC8093AF058EEC41C08091EE
:100EE000D20190E0A0E0B0E082239323A423B523B5
:100EF0000097A105B10539F01092B1058CEA8093F5
:100F0000AF058DEA2DC08091D30190E0A0E0B0E064
:100F100082239323A423B5230097A105B10539F0BB
:100F20001092B10584EC8093AF0585EC19C0109246
:100F3000B1058EEA8093AF058FEA8093B00580916A
:100F4000E2019091E301A091E401B091E5018223D7
:100F50009323A423B5230097A105B10519F089E8CF
:100F60008093B00580911D028823C9F1609192029F
:100F700070919302CB018070907C8050904C79F5F9
:100F80007170DB01A153BC4FEFEAF5E002C08D9315
:100F9000319680818823D9F78091DE019091DF011D
:100FA000A091E001B091E10182239323A423B52312
:100FB0000097A105B10599F08AEE8093AF058BEEFD
:100FC0008093B0051092B105DB01AF52BC4FEFEA40
:100FD000F5E002C08D93319680818823D9F7809106
:100FE0005C01882309F050C06091980270919902C9
:100FF000CB018070907C8050904C09F045C080916E
:10100000D8019091D901A0E0B0E082239323A423DA
:10101000B5230097A105B10511F081E022C08091B0
:10102000DA019091DB01A0E0B0E082239323A423B6
:10103000B5230097A105B10511F082E012C080919F
:10104000EE019091EF01A091F001B091F101282300
:1010500039234A235B232115310541055105A1F0B0
:1010600083E0E82FF0E0EE0FFF1FE559FE4F85917A
:101070009491DB01B170A153BC4F01C02D93FC01D1
:10108000019624912223D1F7089520917F03309176
:1010900080038091820390E02817390720F4809123
:1010A0005C01882339F580917C0290917D028070EB
:1010B000907C8050904CF1F48FEB8093AF05C90188
:1010C00060EB75E044E023E00E94F60489EA809337
:1010D000B4051092B505E0917C02F0917D02F170AB
:1010E000E253FC4FAFEAB5E002C0819311968C91B8
:1010F0008823D9F7089580912902882309F458C0DC
:1011000080916A0290916B028050924008F450C026
:1011100080911C03882311F1E0916D03F0916E031F
:10112000CF016CE370E00E94B1389B0180913702DF
:1011300090E06817790720F080915C018823C1F561
:101140008EE0E031F80728F48CE98093AF05BF0109
:1011500019C081E78093AF05B90114C060916B039A
:1011600070916C032EE06031720720F48BE980935C
:10117000AF0508C080E78093AF05CB016CE370E05A
:101180000E94B13880E090E040EB55E020E00E9402
:10119000C305E0916A02F0916B02F170E153FC4FDC
:1011A000AFEAB5E002C0819311968C918823D9F7FC
:1011B0000895EF92FF920F931F93E0906F03F090CA
:1011C0007003009171031091720360918B03709111
:1011D0008C0380E090E00E94DE369B01AC01C801E8
:1011E000B7010E94D237181644F4C801B7010E9413
:1011F000B23670938C0360938B0380917E02909142
:101200007F028070907C8050904C01F5C801B7013E
:101210000E94AD36DC01CB016FEA75E045E024E0C9
:101220000E94F6048AE98093B4051092B505E09116
:101230007E02F0917F02F170E153FC4FAFEAB5E01E
:1012400002C0819311968C918823D9F71F910F9139
:10125000FF90EF900895CF92DF92EF92FF920F935D
:101260001F93CF93DF93C0909A02D0909B02C60148
:101270008070907C8050904C09F06DC0809113027A
:101280006091350370913603882349F480E090E043
:101290000E94DE362CEB34E743E15DE308C080E0DA
:1012A00090E00E94DE362DED3FE347EB5CE30E94C9
:1012B000D6370E94B236EB016115710519F4C7EEFD
:1012C000D3E02BC060917D0370917E0380E090E0BD
:1012D0000E94DE3620916F033091700340917103BC
:1012E000509172030E94D6377B018C01BE0123E02E
:1012F000660F771F2A95E1F7CC0FDD1F6C0F7D1F5E
:1013000080E090E00E94DE369B01AC01C801B7018D
:101310000E9445360E94B236EB01CE0160EB75E0CB
:1013200044E023E00E94F60480E28093AF058AE265
:101330008093B4051092B505C75ED34060F4D60122
:10134000B170A153BC4FEFEAF5E002C08D93319626
:1013500080818823D9F7DF91CF911F910F91FF9062
:10136000EF90DF90CF90089580915E0290915F02A0
:101370008070907C8050904CC1F580911102882340
:10138000A1F12091A5063091A60680911202882332
:1013900089F037FF02C028593E4FC9016FEA75E056
:1013A00043E020E00E94F6048DEB8093B20510929A
:1013B000B3050CC0C9016FEA75E044E020E00E946B
:1013C000F6048DEB8093B3051092B405E0915E02B4
:1013D000F0915F02F170E153FC4FAFEAB5E002C05B
:1013E000819311968C918823D9F7089520E030E0FD
:1013F00040E450E0F901EE0FFF1FE85CFE4F8591DD
:101400009491DA01A153BC4F01C06D93FC01019688
:1014100064916623D1F72F5F3F4F425E5F4F2830C4
:10142000310541F720E030E0F901E155FA4FD901EB
:10143000A85CBD4F8C9180832F5F3F4F2A303105D0
:1014400099F71092B905EFEAF5E0A7ECB4E002C015
:101450008D93319680818823D9F780917901E82F87
:10146000F0E0EE0FFF1FE85BFE4F85919491A5EE33
:10147000B4E001C02D93FC01019624912223D1F701
:1014800080914203882351F0E3E4F3E0A1E2B5E068
:1014900002C08D93319680818823D9F70895809179
:1014A0002403882359F18091580290915902807049
:1014B000907C8050904C11F5809110028823F1F0BF
:1014C00080913B0390913C036FEA75E043E020E09C
:1014D0000E94F6048DEB8093B2051092B305E09163
:1014E0005802F0915902F170E153FC4FAFEAB5E0B8
:1014F00002C0819311968C918823D9F70895809129
:101500002403882309F445C0E0915202F09153026C
:10151000CF018070907C8050904CD9F58091200351
:1015200090912103A0912203B09123030397A10579
:10153000B10520F480915C01882359F58091A506BE
:101540009091A606845E9D4F20913B0330913C0311
:10155000821B930B880F991F880F991F8D966AE540
:1015600070E00E94C538CB0160E170E00E94C53890
:10157000805A8093AF051092B005DF01B170A1537E
:10158000BC4FEFEAF5E002C08D933196808188234D
:10159000D9F7089520910A012A3069F480910B014E
:1015A000813009F4A1C0823019F0EAE7F1E09EC071
:1015B000E0E7F1E09BC02A3008F096C090910C0162
:1015C000913029F0EAE6F1E0923011F51DC02830A3
:1015D00019F48AE080930A0180910A01893019F494
:1015E00087E080930A0190910A018EE1989FF001B3
:1015F000112480910B0126E0829FC0011124E80F85
:10160000F91FE05CFF4F72C083E080930B0104C0C0
:10161000933071F490930B01283019F48AE0809391
:101620000A0180910A01893009F055C087E051C054
:10163000943079F483E080930B01273019F48AE029
:1016400080930A0180910A01893009F044C086E044
:1016500040C0953041F483E080930B01293019F5A7
:1016600090930A0120C09630A1F4293049F480916A
:101670008101883011F48AE001C088E080930A017A
:1016800080910A018093810193E090930B019EE188
:1016900025C0973069F483E080930B01293019F459
:1016A00085E080930A0180910A018630A1F410C080
:1016B0009830E1F483E080930B0180910A01893036
:1016C00019F487E080930A0180910A01883019F4A7
:1016D0008AE080930A0190910A018EE1989FF001BF
:1016E0001124EE5AFF4F02C0EAE6F1E080915D015D
:1016F000882321F0E153FC4F83E08083089580919B
:1017000042038823B1F08250823020F080915C0146
:10171000882379F0A3E4B3E0E0916C02F0916D02CC
:10172000F170E153FC4F02C0819311968C91882394
:10173000D9F70895CF93DF938091A306982F9F5FE9
:1017400042E056E0FA01E80FF11D208130E0692FF8
:101750006F5FFA01E90FF11D908180E0822B932BDE
:10176000A0E0B0E0262F2F5FFA01E60FF11D6081A7
:1017700070E0420F511DEA01E8812F5F2093A3061C
:101780003E2F20E0262B372B40E050E0A9013327E5
:101790002227282B392B4A2B5B2BB901CA01DF9159
:1017A000CF91089581E080930C018AE080930A0133
:1017B00083E080930B011092880110921D038091A9
:1017C0001902882301F110928D0310928E0310925A
:1017D0008F03109290031092870310928803109247
:1017E000890310928A031092860310928503109247
:1017F00084031092830310928C0310928B03109237
:101800009203109291030E9498030895EF92FF9221
:101810000F931F93CF93DF939091860182E5989F5A
:10182000700111248AE590E0E80EF91EC0E5D2E0CF
:1018300081EB96E0B7010E946B3188831982B70172
:101840006F5F7F4F81EB96E00E946B31182F00E0B5
:1018500028813981200F311F398328838091140218
:10186000882391F0C90191708739910568F0225E53
:101870003F4F398328832E513040813F910520F01E
:10188000245C3F4F3983288382E090E0E80EF91E04
:10189000229692E0C23AD90759F6DF91CF911F9173
:1018A0000F91FF90EF9008955E9A2A9864E670E099
:1018B00080E090E00E94FA312A9A80E58CBD81E0B8
:1018C0008DBD8DB58EB56AE070E080E090E00E943D
:1018D000FA315E9864E670E080E090E00E94FA31B0
:1018E00080EA8EBD0DB407FEFDCF8EB58FEF8EBDA5
:1018F0000DB407FEFDCF9EB59370913029F49093FF
:101900001402909379010CC0923029F410921402C1
:101910001092790105C0809114028E5F8093790145
:101920009093D50580911402882341F080EE91E0D8
:101930009093D4058093D3058CE407C086E891E0AA
:101940009093D4058093D3058CE01EBC0DB407FEA4
:10195000FDCF9EB58EBD0DB407FEFDCF8EB55E9A50
:101960009FB7F894E89A809169008260809369003B
:101970009FBF0E94060C08955E9880EA8EBD0DB44C
:1019800007FEFDCF8EB58FEF8EBD0DB407FEFDCFE8
:101990008EB583709091D505981719F00E94540C5C
:1019A000089580E88EBD0DB407FEFDCF8EB58FEF94
:1019B0008EBD0DB407FEFDCF0EB403FC02C00E9425
:1019C000540C0895EF92FF920F931F93CF93DF93E0
:1019D000C0E0D0E081EB96E0BE010E946B31FE01D9
:1019E000EA50FE4F80832196CC34D10599F772E4FA
:1019F000E72E72E0F72E0CE410E081EB96E0B801E0
:101A00000E946B31F701808311820F5F1F4F81EBC2
:101A100096E0B8010E946B31D82FC0E0F7018081B9
:101A200091818C0F9D1F819391937F010F5F1F4FB9
:101A30000A35110511F70E94060CDF91CF911F9115
:101A40000F91FF90EF9008951F9380916C029091F9
:101A50006D028070907C8050904C09F0BCC08091E9
:101A60000602882309F4B7C080914203882309F055
:101A7000B2C080911C03882349F480919303826053
:101A8000809393038EE18093080117C09091080121
:101A9000992371F080915D01882309F09CC08091A9
:101AA000930384608093930391509093080105C041
:101AB000809193038160809393038091810390E0F0
:101AC00020917D0330917E038217930728F0809147
:101AD00093038064809393038091120383FF1CC05F
:101AE00080913D03853028F4809193038062809338
:101AF000930380916B01882329F480919303806183
:101B00008093930380916A01882331F48091930339
:101B100088608F7C8093930380919403882321F4C1
:101B2000809193038093940380919403182F1195CF
:101B300018230E94C63120917201309173014091A7
:101B40007401509175012C503E4F4F4F5F4F261737
:101B500037074807590798F490919403992329F07F
:101B6000812F80958923809394030E94C6316093CE
:101B7000720170937301809374019093750120E05A
:101B800030E0412F50E0CA01022E02C095958795A2
:101B90000A94E2F780FD622F2F5F3F4F2730310517
:101BA00091F7809193038230B0F0E62FF0E0EE0FD2
:101BB000FF1FEA57FF4F85919491A0916C02B0915D
:101BC0006D02B170A153BC4F01C02D93FC01019671
:101BD00024912223D1F71F9108955F926F927F92F3
:101BE0008F929F92AF92BF92CF92DF92EF92FF922D
:101BF0000F931F93CF93DF935C01EB01809123023E
:101C0000882329F480912B02882309F4C7C080918E
:101C10001C03882321F4109236031092350320917F
:101C20003503309136034091390350913A03CA018C
:101C30000F9682179307F0F40E94C63160936303F6
:101C400070936403809365039093660382E08093AE
:101C50006103809135039091360390933A0380930A
:101C6000390380911001815080931001803130F54B
:101C700085E122C0215F3F4F24173507F8F40E9409
:101C8000C6316093630370936403809365039093FC
:101C9000660381E080936103809135039091360360
:101CA00090933A0380933903809110018F5F809362
:101CB0001001863118F080E1809310012091A2027A
:101CC0003091A3024091A4025091A502E090A60297
:101CD000F090A7020091A8021091A902D801C701B3
:101CE0004496A11DB11D82179307A407B50734F5CB
:101CF0000E94C63160936703709368038093690301
:101D000090936A0382E0809362038091A202909193
:101D1000A302A091A402B091A5028093A602909381
:101D2000A702A093A802B093A9028091110181504B
:101D300080931101803190F585E12EC02C5E3F4FDC
:101D40004F4F5F4F2E153F05400751073CF50E944E
:101D5000C63160936703709368038093690390931F
:101D60006A0381E0809362038091A2029091A302B2
:101D7000A091A402B091A5028093A6029093A7021D
:101D8000A093A802B093A902809111018F5F809364
:101D90001101863118F080E18093110180912302B6
:101DA000882329F483E180931001809311018091AD
:101DB000820290918302BFEFEB2EB1E0FB2EE8226E
:101DC000F922C93CD1051CF0C8ECD0E006C02FEFC9
:101DD000C833D20714F4C8E3DFEF31E9A31631E0CA
:101DE000B3062CF0A0E9AA2EA1E0BA2E09C040E764
:101DF000A4164EEFB40624F4F0E7AF2EFEEFBF2E8C
:101E0000BE01665F7F4F20E030E08070907C8050A4
:101E1000904C11F421E030E08091160290E02823EC
:101E20003923232B09F46EC0CB0168E070E00E94D7
:101E3000C538CC24DD24C61AD70A89E290E0C80E42
:101E4000D91E5090280240E0E4E06E2E712C74E818
:101E5000872E7FEF972E8E0C9F1C443009F445E0AF
:101E6000E42FF0E0C3018E1B9F0B9C012A9DC00153
:101E70002B9D900D3A9D900D112460E470E00E941E
:101E8000C5388B010C0D1D1D0235110568F5E401E7
:101E9000CE0FDF1FC80169E070E00E94C538CB019A
:101EA0009B0165E0220F331F6A95E1F7880F991FA8
:101EB000281B390BC20FD31FC80169E070E00E94D4
:101EC000C538982F9058C153DC4F9883552061F046
:101ED000842F8250853040F4FE01EA55F040908313
:101EE000FE01E65AFF4F90834F5F493008F4B5CFAB
:101EF00080919402909195028070907C8050904CDB
:101F000009F0D3C080911702882309F4D9C08091C9
:101F10008402909185028070907C8050904C09F0F2
:101F2000CFC080918802182F1F70212F21954091DA
:101F300010013091110180918A028F70C82FDD2726
:101F4000C7FDD0958EE12802C0011124D701AC1B3A
:101F5000BD0BA80FB91FA153BC4FFE01EE0DFF1D15
:101F6000E80FF91FE153FC4F4C9330832F5F5E96CF
:101F70007E961217CCF7F701EC1BFD0BE053FC4FDC
:101F800083E08083FE01EE0DFF1DE253FC4F82E0F3
:101F9000808380912B02882309F492C0809186026D
:101FA000909187028070907C8050904C09F088C09E
:101FB0000E94C63120916303309164034091650310
:101FC0005091660328513C4F4F4F5F4F6217730784
:101FD0008407950758F580916103212F332727FD4A
:101FE0003095823089F482EE9FEF289FF001299F7F
:101FF000F00D389FF00D1124EE0DFF1DEC1BFD0BB5
:10200000E153FC4F89EC11C0F90185E0EE0FFF1F91
:102010008A95E1F7220F331FE21BF30BEE0DFF1D34
:10202000EC1BFD0BE153FC4F8FEC80830E94C6310B
:1020300020916703309168034091690350916A03CE
:1020400028513C4F4F4F5F4F621773078407950726
:10205000B8F580916203212F332727FD3095823018
:1020600089F482EE9FEF289FF001299FF00D389FA1
:10207000F00D1124EE0DFF1DEC0FFD1FE153FC4F81
:1020800089EC11C0F90115E0EE0FFF1F1A95E1F779
:10209000220F331FE21BF30BEE0DFF1DEC0FFD1F94
:1020A000E153FC4F8FEC80830BC0F701E153FC4FF1
:1020B00086E2829331968CEB81838EE7808322CFF8
:1020C000DF91CF911F910F91FF90EF90DF90CF9014
:1020D000BF90AF909F908F907F906F905F9008958A
:1020E000CF93DF93C0E0D0E081EB96E0BE0140E00B
:1020F0000E947231219682E0C030D807A9F7DF91A3
:10210000CF910895CF92DF92EF92FF920F931F939A
:10211000CF93DF9381EB96E060E070E00E946B313B
:102120008C3009F476C0C0E0D0E0FE01ED58FE4FDF
:10213000E49181EB96E0BE014E2F0E947231219610
:10214000CC34D10591F7EE24FF24CCE4D0E0F701A4
:10215000EE0FFF1FE154FE4F0591149181EB96E0C5
:10216000BE01402F0E947231219681EB96E0BE01A4
:10217000412F0E9472310894E11CF11C219687E0E6
:10218000E816F10421F7CC24DD24CAE5D0E076017D
:10219000EE0CFF1CF701E353FE4F0591149181EB08
:1021A00096E0BE01402F0E947231219681EB96E0AD
:1021B000BE01412F0E947231F701E15EFD4FE590B3
:1021C000F490CF5ADF4F81EB96E0BE014E2D0E9476
:1021D0007231219681EB96E0BE014F2D0E94723143
:1021E000CF5ADF4F81EB96E0BE01402F0E94723143
:1021F000219681EB96E0BE01412F0E947231089436
:10220000C11CD11CC35AD04082E5C816D10409F0C4
:10221000BECFDF91CF911F910F91FF90EF90DF9094
:10222000CF9008950F931F93CF93DF93C0E0D0E03A
:10223000FE01EA50FE4F81EB96E0BE0140810E9414
:1022400072312196CC34D10599F702E412E0CCE446
:10225000D0E081EB96E0BE01F80140810E9472312E
:102260002196F801418181EB96E0BE010E94723116
:102270000E5F1F4F2196F2E000351F0751F781EBEB
:1022800096E060E070E04CE00E947231DF91CF9107
:102290001F910F91089583E497E06091A7060E9433
:1022A000193508951F93182F83E497E0612F0E943A
:1022B00019358091A70681278093A7061F9108955D
:1022C0001F93192F0E945211812F0E9452111F91AA
:1022D00008950F931F93082F162F83E497E064E26D
:1022E0000E94193583E497E06DE40E94193583E478
:1022F00097E06CE30E9419351092A706812F0E9487
:102300005211802F0E945211112311F40E944B117F
:102310001F910F9108958CED63E00E94691189E08F
:102320000E9452118091C3019091C4010E946011DA
:102330000E944B1108951F938CED6FE10E9469116B
:1023400089E00E94521110E06091C3017091C401B4
:1023500081EB96E00E946B318093C5018091C301AF
:102360009091C4010E9460118091C5010E94521198
:102370008091C3019091C40101969093C401809310
:10238000C3011F5F1A3001F70E944B111F9108957E
:10239000CF93DF938091D7058093D8058AEC6EE1C7
:1023A0000E946911C0E0D0E0FE01E752FA4F80813F
:1023B0000E945211FE01ED51FA4F80810E9452118C
:1023C000FE01E351FA4F80810E9452112196CA30DA
:1023D000D10551F70E944B118CEC67E00E94691106
:1023E0008091F7050E9452118091F8050E945211C8
:1023F0008091F9050E9452118091FA050E945211B4
:102400008091FB050E9452118091FC050E9452119F
:102410008091FD050E9452110E944B110E941211E1
:102420008AEF60E00E9469110E94D20BDF91CF9188
:10243000089520910A012A30C9F480910B0183305C
:10244000A9F480917A0182301CF081E080937A01B6
:1024500080917A018F3F1CF48FEF80937A018091F5
:102460000C0190917A01890F80930C0180910C01ED
:1024700087FF03C088E080930C0180910C018930B4
:1024800014F010920C0130910C01313011F5E22F53
:10249000E150E73008F06BC2263008F0EE5F809123
:1024A0000B01823049F0833081F0813009F05FC246
:1024B000F0E0E752FA4F03C0F0E0ED51FA4F8081AF
:1024C00090917A01890F808352C2F0E0E351FA4F74
:1024D000F6CF323009F051C080910B01833009F002
:1024E00046C2243051F1253040F42230B1F023307F
:1024F000E0F4213009F03BC208C0263071F12630EB
:1025000020F1273009F033C230C08091F705909157
:102510007A01890F8093F70508958091F8059091CD
:102520007A01890F8093F80508958091F9059091BB
:102530007A01890F8093F9051AC28091FA0590916A
:102540007A01890F8093FA0508958091FB05909197
:102550007A01890F8093FB050AC28091FC05909156
:102560007A01890F8093FC0508958091FD05909173
:102570007A01890F8093FD050895333009F054C026
:1025800080910B01833009F0F2C1243059F12530DC
:1025900040F42230B9F02330E8F4213009F0E7C1EB
:1025A00008C0263081F1263030F1273009F0DFC134
:1025B00032C090E08091FD01882309F491E090936E
:1025C000FD01089580917A0190910002890F809316
:1025D0000002089580917A019091FE01890F809305
:1025E000FE01C5C190E080910702882309F491E0C3
:1025F00090930702089580917A0190910802890FC3
:1026000080930802B4C180917A019091FF01890FF3
:102610008093FF01089590E080910102882309F4DE
:1026200091E0909301020895343009F056C08091F2
:102630000B01833009F09BC12330E9F0243030F4E2
:10264000213061F0223009F092C111C0253029F10A
:102650002530D0F0263009F08AC12FC090E080915B
:10266000FA01882309F491E09093FA0108958FE02C
:1026700080936001089590E08091FB01882309F424
:1026800091E09093FB01089590E08091FC018823F4
:1026900009F491E09093FC016AC180917A01992735
:1026A00087FD909520914A0230914B02820F931F33
:1026B00090934B0280934A02089580917A01992762
:1026C00087FD90952091480230914902820F931F17
:1026D00090934902809348020895353009F050C024
:1026E00080910B01833009F042C1233001F1243085
:1026F00030F4213051F0223009F039C10FC02430BC
:10270000F9F0253009F033C12BC090E0809102022E
:10271000882309F491E090930202089590E080915B
:102720000402882309F491E090930402089590E054
:1027300080910502882309F491E0909305020895A1
:1027400080917A01992787FD9095209146023091DA
:102750004702820F931F9093470280934602089589
:1027600080917A01992787FD9095209144023091BC
:102770004502820F931F909345028093440208956F
:10278000363009F062C080910B01833009F0EFC050
:10279000243079F1253040F42230C9F0233000F59F
:1027A000213009F0E4C00AC02630A9F1263050F1EA
:1027B0002730D1F1283009F0DAC03FC090E0809195
:1027C0001602882309F491E090931602089590E090
:1027D00080911702882309F491E0909317020895DD
:1027E00090E080912302882309F491E090932302E2
:1027F000BEC090E080911502882309F491E0909387
:102800001502089590E080910D02882309F491E06B
:1028100090930D02ACC090E080912A02882309F4C5
:1028200091E090932A02089590E0809124028823F9
:1028300009F491E090932402089580917A01909197
:102840001A02890F80931A0208953730E1F58091BA
:102850000B01833009F08BC0233001F1243030F4B8
:10286000213051F0223009F082C00FC02430F9F03D
:10287000253009F07CC01FC090E0809113028823AE
:1028800009F491E090931302089590E080911B0267
:10289000882309F491E090931B02089590E08091C1
:1028A0002202882309F491E09093220208958AE09D
:1028B00080936101089580917A0190913002890F8F
:1028C000809330020895383009F051C080910B0197
:1028D000833009F04CC0243049F1253040F42230D7
:1028E000A9F02330D8F4213009F041C007C02630C8
:1028F00069F1263018F12730D1F530C080917A0186
:1029000090913402890F80933402089580917A0166
:1029100090913502890F80933502089580917A0154
:1029200090913602890F80933602089580917A0142
:1029300090913702890F80933702089580917A0130
:1029400090910A02890F80930A02089580917A017A
:1029500090910B02890F80930B02089590E0809173
:102960000602882309F491E09093060208952A3024
:1029700071F430930D0180910B01813019F0823098
:1029800031F403C00E94D20B08950E94C81108952B
:102990001F93CF93DF9380911F0190912001855168
:1029A00095408F589140E8F480911D0190911E014F
:1029B00035E085319307A8F0845A964090F48091D1
:1029C00021019091220135E08531930750F0845A1E
:1029D000964038F41092A20688EE93E0A0E0B0E0B2
:1029E00025C08091A206813049F50E94C631209110
:1029F0009E0630919F064091A0065091A106621B51
:102A0000730B840B950B20919A0630919B06409195
:102A10009C0650919D06261737074807590710F462
:102A20001092A2068CE291E0A0E0B0E080939A06BA
:102A300090939B06A0939C06B0939D068091A2065E
:102A4000882309F0E5C0C0911F01D091200137E033
:102A5000CB33D30760F180912101909122018B53F8
:102A6000974028F180912301909124018F57944041
:102A7000F0F080918801882309F0BCC080917B012F
:102A800090917C01069708F4B5C080911C038823BF
:102A900009F0B0C082E08093A20681E080938801B3
:102AA00080910D0180930C010E949803A3C0809136
:102AB0008801882309F49EC010917A0110927A014E
:102AC00080911D03882361F080912301909124015E
:102AD0008551954028F082E08093A2060E94D20B97
:102AE00020918801222309F44FC080911D0190910B
:102AF0001E0137E08B33930778F081E08093A206C4
:102B000080910B018F5F80930B01843008F472C0B9
:102B100083E080930B016EC08E57944070F491E077
:102B20009093A20680910B01815080930B01882322
:102B300009F060C090930B015DC087E0CB33D807EC
:102B400090F091E09093A20680910A0181508093C9
:102B50000A01882311F490930A0180910C018823C3
:102B600009F048C00DC0CE57D44070F481E0809386
:102B7000A20680910A018F5F80930A018B30D0F109
:102B80008AE080930A0136C080911D03882391F565
:102B9000222381F1812F16300CF085E0282F8B3F06
:102BA0000CF42BEF809121019091220134E08E37BB
:102BB000930738F481E08093A206215020937A0194
:102BC00017C08B539740B0F081E08093A2062F5F2F
:102BD00020937A0180910C01883051F480910B018F
:102BE000833031F480910A01853011F41092610133
:102BF0000E9419128091A206813051F40E94C631C0
:102C000060939E0670939F068093A0069093A10602
:102C1000DF91CF911F9108950F931F93CF93DF936F
:102C200080916E0190916F01019690936F01809356
:102C30006E011092A30683E080936A0180910006E2
:102C40008C3D09F026C12091020611E01093A306E5
:102C5000293029F5209104068091030690E0820F27
:102C6000911D9093C4018093C3019091050684E067
:102C70008093A3069093C5011093C6010E94C631AC
:102C80006854744F8F4F9F4F6093C7017093C80172
:102C90008093C9019093CA010E949B11FAC0283009
:102CA00009F05FC010E001E0A091A306EA2FEF5FFA
:102CB0002E2F2F5FF0E0EE5FF94FD081C0E0B0E043
:102CC000AE5FB94F8C91AE01480F511D5093C401B6
:102CD0004093C301E22FF0E0EE5FF94F80812F5F58
:102CE0002093A3068093C5010093C6010E94C631BC
:102CF0006854744F8F4F9F4F6093C7017093C80102
:102D00008093C9019093CA016091C3017091C4017D
:102D100081EB96E04091C5010E94723181EB96E013
:102D200060E070E04CE00E9472318091C3019091AC
:102D3000C4018A35910519F08055914011F40E9423
:102D4000E20C1F5F1A3009F0AFCF8091C301909160
:102D5000C40101969093C4018093C3010E948B111A
:102D600098C02730D9F58CED6BE00E94691187E09F
:102D70000E945211CEEBD2E088819981F3E09695C2
:102D80008795FA95E1F70E946011649683E0C2325C
:102D9000D80791F70E944B118CED6DE00E946911EC
:102DA0008AE00E94521184E090E00E94601181E06C
:102DB00090E00E94601182E796E00E94601181E03D
:102DC00090E00E94601180E090E00E94601181E03C
:102DD00090E00E9460110E944B115BC0233009F00B
:102DE0004DC05091FE05553061F58091030690E08D
:102DF000409104062093A306342F20E0282B392B82
:102E000020523D4109F045C0809105068093C001E4
:102E1000809106065093A3068093C10180911C0304
:102E20008823B9F580918801882399F580918901DB
:102E3000882379F580E88093C20181E0809389013D
:102E400028C0583331F5AAE8B1E091E0E92FF0E06D
:102E5000EE5FF94F80818D939F5F21E0A03CB20728
:102E6000A9F71091390688E38093A306812F0E9469
:102E700095041F3F71F40E94540C0BC0263029F4B6
:102E80000E9470100E94821002C0253011F410932D
:102E9000780180910006843681F481E08093760188
:102EA0008091A306E82FF0E0EE5FF94F90818F5FED
:102EB0008093A3069093180399C0853609F074C0D7
:102EC000E091A306AE2FAF5FF0E0EE5FF94F2081F7
:102ED00030E04A2F4F5FB0E0AE5FB94F9C9180E089
:102EE000822B932B90937E0180937D01E42FEF5FE3
:102EF000A42FB0E0AE5FB94F2C9130E0AE2FAF5FA2
:102F0000F0E0EE5FF94F908180E0822B932B90935D
:102F1000800180937F018A2F8F5FB0E0AE5FB94F51
:102F20002C9130E0E82FF0E0EE5FF94F40818F5FA9
:102F30008093A306942F80E0822B932B909313030E
:102F4000809312030E949A0B6093140370931503ED
:102F5000809316039093170310921C032091D101C4
:102F600030E040E050E02623372348235923211541
:102F700031054105510519F081E080931C038091D2
:102F8000A306E82FF0E0EE5FF94FE0818F5F8093BA
:102F9000A306E093D70580918801882339F5E09353
:102FA000D805E093A40622C0893601F53091A30626
:102FB000ADE1B1E0232FE22FF0E0EE5FF94F808129
:102FC00090E02F5FE22FF0E0EE5FF94FF081E0E05C
:102FD0008E2B9F2B8D939D932F5F41E0AD32B407D5
:102FE00051F7305F3093A3060E94C8148091000609
:102FF0008A3609F09FC085E080936B01E091A306BB
:103000009E2F9F5FF0E0EE5FF94F8081882319F0DB
:1030100081E080932403E92FF0E0EE5FF94F808197
:103020009F5F9093A30680933D030E949A0B609349
:1030300025037093260380932703909328030E940F
:103040009A0B6093290370932A0380932B03909328
:103050002C03E091A306AE2FAF5FF0E0EE5FF94FD7
:10306000208130E0EA2FEF5FB0E0AE5FB94F9C9176
:1030700080E0822B932B9C0140E050E020932D03B5
:1030800030932E0340932F035093300380911C0301
:10309000882341F420933103309332034093330368
:1030A0005093340380912D0390912E03A0912F0310
:1030B000B0913003209131033091320340913303BA
:1030C00050913403821B930BA40BB50B80932D03FB
:1030D00090932E03A0932F03B0933003AE2FAF5FD6
:1030E000F0E0EE5FF94F208130E04A2F4F5FB0E013
:1030F000AE5FB94F9C9180E0822B932B9093360367
:1031000080933503E42FF0E0EE5FF94F20814F5FAD
:1031100030E0E42FF0E0EE5FF94F50814F5F4093D5
:10312000A306952F80E0822B932B909338038093F6
:10313000370314C38B36A9F5E091A3068E2F8F5F5A
:10314000F0E0EE5FF94F208130E0482F4F5FE82F2D
:10315000F0E0EE5FF94F908180E0822B932BA0E0AE
:10316000B0E08093200390932103A0932203B093B7
:103170002303E42FF0E0EE5FF94F20814F5F30E052
:10318000E42FF0E0EE5FF94F50814F5F4093A306CC
:10319000952F80E0822B932B90933C0380933B03ED
:1031A000DDC28C3609F04EC04091A306842F8F5F9C
:1031B000E42FF0E0EE5FF94F208130E0A82FAF5F01
:1031C000E82FF0E0EE5FF94F908180E0822B932BA7
:1031D0009093AB028093AA02EA2FF0E0EE5FF94FE2
:1031E000208130E0AF5FB0E0AE5FB94F9C9180E0EE
:1031F000822B932B9093AD028093AC024C5FE42F13
:10320000F0E0EE5FF94F80814F5F682F70E0E42FB0
:10321000F0E0EE5FF94F20814F5F4093A306922FBD
:1032200080E0682B792B7093A6066093A506643B1B
:1032300071050CF493C2685671407093A6066093B2
:10324000A5068CC28D3621F50E949A0B6093A202CE
:103250007093A3028093A4029093A5028091A30689
:10326000E82FF0E0EE5FF94F20818F5F30E0E82F2C
:10327000F0E0EE5FF94F40818F5F8093A306942FBB
:1032800080E0822B932B90931B0380931A0366C2DA
:103290008E3609F04AC0E091A306AE2FAF5FF0E092
:1032A000EE5FF94F808180931903EA2FEF5FB0E062
:1032B000AE5FB94F2C9130E0AE2FAF5FF0E0EE5F24
:1032C000F94F908180E0822B932B90933F03809362
:1032D0003E03EA2FEF5FB0E0AE5FB94F2C9130E0D4
:1032E0004E2F4F5FF0E0EE5FF94F908180E0822B30
:1032F000932B9093410380934003E42FF0E0EE5F23
:10330000F94F20814F5F30E0E42FF0E0EE5FF94F9E
:1033100050814F5F4093A306952F80E0822B932B23
:10332000909378038093770319C28F3609F046C0D3
:10333000E091A306AE2FAF5FF0E0EE5FF94F808122
:103340008093F705EA2FEF5FB0E0AE5FB94F8C9145
:103350008093F805AE2FAF5FF0E0EE5FF94F80810C
:103360008093F905EA2FEF5FB0E0AE5FB94F8C9123
:103370008093FA059E2F9F5FF0E0EE5FF94F80810A
:103380008093FB05E92FF0E0EE5FF94F80819F5FAE
:103390008093FC05E92FF0E0EE5FF94F80819F5F9D
:1033A0009093A3068093FD058091C3059091C40579
:1033B000A091C505B091C6059D7F6FC08537B9F551
:1033C000A7E9B3E03091A30620E097E040E01FC0FA
:1033D000E32FF0E0EE5FF94FE081822F85508230DD
:1033E00088F0293078F4EB3341F41C92892F90E077
:1033F0000196A80FB91F97E007C0992331F0ED930C
:10340000915003C0EB3309F42F5F4F5F3F5F809112
:10341000FE054817E8F23093A3068091C30590910A
:10342000C405A091C505B091C605AF7D36C08037F3
:10343000E9F54091A306942F20E030E0D901A7528E
:10344000BA4FE92FF0E0EE5FF94F80818C93D901FC
:10345000AD51BA4F9F5FE92FF0E0EE5FF94F8081E9
:103460008C93D901A351BA4F9F5FE92FF0E0EE5F33
:10347000F94F80818C932F5F3F4F9F5F2A3031053A
:10348000E9F6425E4093A3068091C3059091C4057E
:10349000A091C505B091C6059B7F8093C30590930D
:1034A000C405A093C505B093C60558C1823FA1F5D8
:1034B000E091A3063E2F3F5FF0E0EE5FF94F808181
:1034C000809342038091FE0590E08E3191051CF0BF
:1034D000EDE1F0E002C0FC013197ED5BFC4F1082A2
:1034E00020E00EC02D3110F0ADE1B0E0AD5BBC4F7F
:1034F000E32FF0E0EE5FF94F80818C932F5F3F5F09
:10350000A22FB0E08091FE0590E00197A817B907BF
:103510004CF33093A30622C1873709F01FC181E025
:10352000809377010091FE0585E2E1EDF1E0DF0196
:103530001D928A95E9F76091A306102F762F21E05E
:1035400030E040E050E004C1E72FF0E0EE5FF94FDB
:10355000E081EB3009F463C0EC30A4F4E330E9F12E
:10356000E4303CF4E13069F1E2308CF5EE2319F1FE
:10357000E9C0E830F1F1EA3009F446C0E53009F07D
:10358000E1C031C0E43109F48AC0E53154F4E031DE
:1035900009F45BC0E33109F46DC0EC3009F0D2C02E
:1035A00049C0EC3109F4A5C0ED3109F4B7C0E531EB
:1035B00009F0C8C089C08091D101822B8093D101CC
:1035C000C1C08091D201822B8093D201BBC0809177
:1035D000D301822B8093D301B5C08091D401822B7B
:1035E0008093D401AFC08091D501822B8093D50107
:1035F000A9C08091D6019091D701822B932B9093F3
:10360000D7018093D6019EC08091D8019091D901B5
:10361000822B932B9093D9018093D80193C08091F2
:10362000DA019091DB01822B932B9093DB01809345
:10363000DA0188C08091DC019091DD01822B932B0F
:103640009093DD018093DC017DC08091EA0190912F
:10365000EB01A091EC01B091ED01822B932BA42BF7
:10366000B52B8093EA019093EB01A093EC01B0930A
:10367000ED0168C08091E6019091E701A091E80119
:10368000B091E901822B932BA42BB52B8093E601FB
:103690009093E701A093E801B093E90153C08091B2
:1036A000EE019091EF01A091F001B091F101822B18
:1036B000932BA42BB52B8093EE019093EF01A09355
:1036C000F001B093F1013EC08091F2019091F301BD
:1036D000A091F401B091F501822B932BA42BB52B73
:1036E0008093F2019093F301A093F401B093F5015C
:1036F00029C08091DE019091DF01A091E001B0919D
:10370000E101822B932BA42BB52B8093DE019093A8
:10371000DF01A093E001B093E10114C08091E201C8
:103720009091E301A091E401B091E501822B932BEC
:10373000A42BB52B8093E2019093E301A093E401C5
:10374000B093E501220F331F441F551F11507F5FB7
:10375000112309F0F9CE600F6093A306DF91CF919A
:103760001F910F910895CF92DF92EF92FF921F93D6
:10377000CF93DF93182F83E497E00E94AF3420E0CB
:10378000892B09F481C021E07FC083E497E00E9487
:10379000E034382F809170019091710101969093DF
:1037A000710180937001809198069091990600971D
:1037B00061F41092990610929806343209F059C0BB
:1037C000D0939906C093980654C08130910529F48E
:1037D0003D3441F482E090E00AC08230910561F40A
:1037E0003E3319F080E090E002C083E090E09093D7
:1037F0009906809398063DC08330910559F4373976
:1038000058F53093FE05F0929906E09298063093B1
:10381000FF052FC08430910571F4D0929906C092B3
:103820009806309300068091FF0583278093FF055B
:10383000109201061EC00597E1F42091FF05232791
:103840002093FF05909101068091FE05981749F499
:10385000222311F40E940C161092990610929806D9
:1038600008C0E92FF0E0EE5FF94F30839F5F90933F
:10387000010683E497E00E94AF34892B81F0812F09
:10388000111181E0282F08C0B5E0CB2ED12CA4E087
:10389000EA2EF12CC1E0D0E0213009F476CFDF919F
:1038A000CF911F91FF90EF90DF90CF900895EF920E
:1038B000FF920F931F930E94C6317B018C0188E217
:1038C00090E0A0E0B0E0E80EF91E0A1F1B1F81E0A7
:1038D0008093D6050DC00E94C631E616F70608078C
:1038E000190718F41092D60503C080E00E94B31B9C
:1038F0008091D605882379F71F910F91FF90EF9063
:103900000895EF92FF920F931F93CF93DF935E98EA
:1039100085E08EBD0DB407FEFDCF8EB51EBC0DB487
:1039200007FEFDCF8EB586E08EBD0DB407FEFDCF40
:103930008EB51EBC0DB407FEFDCF8EB584E08EBDE6
:103940000DB407FEFDCF8EB581E08EBD0DB407FE30
:10395000FDCF8EB50E94571C0FEC13E0C0E0D0E005
:1039600097E0E92E80E2F82E15C0C03FD10511F492
:103970000E94571CF8018081EEBC0DB407FEFDCFFC
:103980009EB58EBD0DB407FEFDCF8EB5F801F19248
:103990008F0121968091D3059091D405C817D9073E
:1039A00020F387E08EBD0DB407FEFDCF8EB58FEFFF
:1039B0008EBD0DB407FEFDCF8EB584E08EBD0DB477
:1039C00007FEFDCF8EB51EBC0DB407FEFDCF8EB534
:1039D0005E9ADF91CF911F910F91FF90EF90089524
:1039E0000F931F93DC01CB01142F022F642F70E083
:1039F00061557A4F4AE050E00E943E03113059F47D
:103A0000E02FF0E080911302E15CFE4FE80FF11D22
:103A100080818093AF051F910F91089580912403B9
:103A2000882309F462C0809113028823A1F0609179
:103A300020037091210380912203909123030E941F
:103A4000DE3621EA38EF41E550E40E94D6370E9485
:103A5000B236FB0104C0E0912003F09121039F01E5
:103A600040E050E08091870390918803A091890302
:103A7000B0918A0382179307A407B50740F42093F7
:103A80008703309388034093890350938A0380917E
:103A90005402909155028070907C8050904C29F592
:103AA000CF0164E670E00E94B1388091340290E06A
:103AB0006817790720F080915C018823B1F4BF0179
:103AC00080E090E041E022E00E94F01CE09154028E
:103AD000F0915502F170E153FC4FAFEAB5E002C03E
:103AE000819311968C918823D9F7089580911302C0
:103AF0008823A1F06091A2027091A3028091A40298
:103B00009091A5020E94E0362EEA31E646E05DE3A0
:103B10000E94D6370E94AD369B010EC06091A20272
:103B20007091A3028091A4029091A50224E630E056
:103B300040E050E00E94FA3880911C03882389F00D
:103B400080917B0190917C01069758F080918503CC
:103B5000909186038217930724F430938603209371
:103B6000850380916202909163028070907C805006
:103B7000904C59F580912602882339F1C9016AE0F9
:103B800070E00E94C5388091350290E0681779078F
:103B900024F080915C018823C1F4B901882777FD66
:103BA0008095982F41E020E00E94F01CE091620295
:103BB000F0916302F170E153FC4FAFEAB5E002C04F
:103BC000819311968C918823D9F70895EF92FF92F3
:103BD0000F931F9380910F02882309F456C08091A0
:103BE0005A0290915B028070907C8050904C09F05A
:103BF0004CC0809113028823A9F060912D0370912D
:103C00002E0380912F03909130030E94E03621EA29
:103C100038EF41E550E40E94D6370E94AD367B0173
:103C20008C0108C0E0902D03F0902E0300912F032B
:103C300010913003B701C8012AE030E040E050E0C5
:103C40000E94FA388091350290E0A0E0B0E0281799
:103C500039074A075B0724F080915C018823A9F4A7
:103C6000B701C80141E020E00E94F01CE0915A0237
:103C7000F0915B02F170E153FC4FAFEAB5E002C096
:103C8000819311968C918823D9F71F910F91FF9002
:103C9000EF900895CF92DF92EF92FF920F931F93D0
:103CA000CF93DF9380912403882309F481C00E947D
:103CB000E61DC0917202D0917302CE018070907C9B
:103CC0008050904C09F074C0E0901403F0901503FC
:103CD00000911603109117032091D8013091D9015A
:103CE00080E090E0E114F1040105110511F481E098
:103CF00090E082239323892B09F05AC040E050E0E2
:103D00002E213F214023512380910D0290E0A0E01D
:103D1000B0E0282B392B4A2B5B2B211531054105AF
:103D2000510509F445C08AEC8093AF0560912503E5
:103D300070912603809127039091280340EB55E072
:103D400024E00EE4E3E5EE2E0E944C05DE01B170A6
:103D5000A153BC4FEFEAF5E002C08D93319680810C
:103D60008823D9F7C0907402D09075028FEF91E04C
:103D7000C822D9228BEC8093AF0560912903709102
:103D80002A0380912B0390912C0340EB55E024E013
:103D900005E437E5E32E0E944C05D601A153BC4F44
:103DA000EFEAF5E002C08D93319680818823D9F740
:103DB000DF91CF911F910F91FF90EF90DF90CF9007
:103DC00008951F9380912403882309F46AC0809189
:103DD0001C03882321F410923603109235031091AE
:103DE00013026091350370913603112349F480E08A
:103DF00090E00E94DE362CEB34E743E15DE308C03F
:103E000080E090E00E94DE362DED3FE347EB5CE37F
:103E10000E94D6370E94B2362091830330918403EA
:103E2000C90144968617970728F4909384038093DA
:103E3000830307C02617370720F470938403609329
:103E4000830380915602909157028070907C80503D
:103E5000904C39F58091360290E08617970720F450
:103E600080915C018823E9F4E12FF0E0E95BFE4FEB
:103E700080818093AF05CB0160EB75E04AE050E0B4
:103E80000E943E03E0915602F0915702F170E15317
:103E9000FC4FAFEAB5E002C0819311968C91882364
:103EA000D9F71F91089520913D03253020F480918A
:103EB0005C01882331F5809150029091510280700D
:103EC000907C8050904CE9F48EE18093AF058FE1B7
:103ED0008093B005822F90E061EB75E04AE050E0FE
:103EE0000E943E03E0915002F0915102F170E153C3
:103EF000FC4FAFEAB5E002C0819311968C91882304
:103F0000D9F7089580917602909177028070907C25
:103F10008050904C59F58AEB8093AF0580917903DE
:103F200090917A0360EB75E04AE050E00E943E0316
:103F3000E0E0AE2FB0E0A155BA4F8C91EF5F88233F
:103F4000C1F785E28C93F0E0E155FA4F1082E091E1
:103F50007602F0917702F170E253FC4FAFEAB5E0E0
:103F600002C0819311968C918823D9F7089580918E
:103F70008002909181028070907C8050904C51F52D
:103F800084EA8093AF05609173037091740380910C
:103F900075039091760320E030E044EB53E40E94F7
:103FA00045360E94AD36DC01CB0160EB75E04AE09E
:103FB00050E00E943E03E0918002F0918102F17096
:103FC000E153FC4FAFEAB5E002C0819311968C91AA
:103FD0008823D9F708952F923F924F925F926F9264
:103FE0007F928F929F92AF92BF92CF92DF92EF9289
:103FF000FF920F931F93DF93CF93CDB7DEB72E972A
:104000000FB6F894DEBF0FBECDBF80911A0282308A
:1040100059F0833020F4813009F01AC20CC083308B
:1040200089F0843009F014C221E030E042E050E031
:1040300058874F830DC020E030E081E090E0988702
:104040008F8306C020E030E0E2E0F0E0F887EF8305
:1040500080912403882309F4FBC1809194029091FC
:1040600095028070907C8050904C09F0F1C12B83B8
:104070001E821D82E4C120913B0330913C034B81A1
:10408000413071F480911E0390911F03281B390B5E
:10409000C901845E9D4F68E671E00E94B1380EC090
:1040A00028593E4F8091A5069091A606F901E81B7C
:1040B000F90BCF0168E671E00E94C5389C016AE502
:1040C00070E00E94C5386130710589F06230710579
:1040D0001CF4672B41F024C06230710589F0633015
:1040E0007105F1F414C0F1E0FE834FEF18C084EBCA
:1040F00090E0821B930B9C0191E09E839D8310C0F6
:10410000245B3040EFEFEE83F1E0FD8309C088E6E9
:1041100091E06C01C21AD30A96014FEF4E834D8392
:10412000B901882777FD8095982F0E94E0362BED06
:104130003FE049E450E40E94D63720E030E044E319
:1041400053E40E9445367B018C01609120037091FD
:10415000210380912203909123030E94DE365B01AC
:104160006C01B701C8010E9439389B01AC01C6013E
:10417000B5010E94D6370E94B2367A836983B701AF
:10418000C8010E9442369B01AC01C601B5010E94E4
:10419000D6370E94B2367E876D87E981FA81E617AD
:1041A000F70710F41B0103C0C980DA80160144240C
:1041B000552424E6221631044104510428F484E6EF
:1041C00090E031E23C831FC044EF241641E0340606
:1041D00040E0440640E0540628F484EF91E052E2C7
:1041E0005C8311C084EC281689E0380680E048061C
:1041F00080E0580628F484EC99E0E3E2EC8303C005
:10420000C101F4E2FC833C01882477FC8094982C63
:1042100000D000D0C980DA80B60180E090E020E1D3
:1042200030E040E050E0EDB7FEB7218332834383B6
:10423000548320E030E040E050E084017301AA2480
:10424000BB2465010E94553369877A878B879C87D9
:10425000CD84DE84B60180E090E02FE030E040E0E5
:1042600050E0EDB7FEB7218332834383548320E0CF
:1042700030E040E050E0AA24BB2465010E945533A1
:104280007B018C010F900F900F900F90F4E12F168F
:1042900031044104510428F400E010E0AA24BB24B6
:1042A0001AC0CE802C2D332727FD3095432F532F56
:1042B00069857A858B859C850E9485385B01DD80C8
:1042C0002D2D332727FD3095432F532FC801B701DC
:1042D0000E9485388B01E0909602F09097022FEFB4
:1042E00031E0E222F3223B81313011F045E001C0A0
:1042F00044E0C501B7FE04C0882799278A199B09A5
:1043000062E00E94A438292FC80117FF04C0882743
:104310009927801B910B63E00E94A438692F5D816F
:10432000513019F482E0891B682F8E818F3F19F478
:1043300091E0921B292FC8010296059718F461E0BD
:10434000ED816E1BC5010196039728F42B2D209556
:10435000221F2227221FFB81FF2311F030ED01C015
:1043600036ED80911A02843039F083E02802C001D2
:104370001124680F630F15C08091A5069091A606C1
:1043800020911E0330911F03821B930B8A519D4F76
:1043900068E671E00E94B1386DE270E00E94B138C9
:1043A0006E58CC80C092AF051092B005E091940297
:1043B000F0919502F170E153FC4FAFEAB5E002C015
:1043C000219311962C912223D9F76093AF05109277
:1043D000B005C50162E070E00E94C538FB01EE0D3A
:1043E000FF1DC80163E070E00E94C538CB019B014E
:1043F000B5E0220F331FBA95E1F7880F991F281BEC
:10440000390BE20FF31FE153FC4FAFEAB5E002C0F6
:10441000819311968C918823D9F74093AF05109220
:10442000B005D701A153BC4FEFEAF5E002C08D9370
:10443000319680818823D9F72B812F5F2B833B8195
:10444000832F90E04F815885841795070CF413CE85
:104450002E960FB6F894DEBF0FBECDBFCF91DF9181
:104460001F910F91FF90EF90DF90CF90BF90AF9092
:104470009F908F907F906F905F904F903F902F9084
:104480000895AF92BF92CF92DF92EF92FF920F9377
:104490001F93CF93DF93E0916402F0916502CF0107
:1044A0008070907C8050904C09F062C08091250211
:1044B000882309F45DC0EF01D170FE01E153FC4F88
:1044C0007E978FE780837E968083868F20911A0364
:1044D00030911B032937310514F068E705C0622FBE
:1044E00028583F4F0CF468E800D000D0772767FDCC
:1044F0007095872F972F21E130E040E050E0EDB735
:10450000FEB7218332834383548328E730E040E0C1
:1045100050E0E8E8EE2EEFEFFE2EEFEF0E2FEFEF7C
:104520001E2FAA24BB2465010E945533262F862FF7
:1045300066E00E94A4388150992787FD9095FC0180
:1045400045E0EE0FFF1F4A95E1F7880F991FE81B22
:10455000F90BEC0FFD1FE153FC4F822F66E00E9428
:10456000A4388FE8891B80830F900F900F900F90D5
:10457000DF91CF911F910F91FF90EF90DF90CF903F
:10458000BF90AF900895AF92BF92CF92DF92EF921B
:10459000FF920F931F938091660290916702807043
:1045A000907C8050904C09F08BC080E28093B005E5
:1045B0006091230170912401809114019091150163
:1045C0008617970720F4709315016093140180916A
:1045D0001201909113016817790720F47093130169
:1045E00060931201809114019091150183509840BD
:1045F00030F082E098E0909315018093140180914F
:10460000120190911301865B934030F486EB93E0A6
:10461000909313018093120180911C03882369F405
:1046200090E29093B0059093B1058DE28093B2052E
:104630008093B3059093B4052FC000D000D080E0E4
:1046400090E0209112013091130140E050E0E090A1
:104650001401F090150100E010E0F4E6AF2EB12C4B
:10466000C12CD12CEDB7FEB7A182B282C382D48215
:10467000AA24BB2465010E945533DC01CB010F90B5
:104680000F900F900F9061EB75E043E020E00E94E7
:10469000F60485E28093B40588EC8093AF05109210
:1046A000B505E0916602F0916702F170E153FC4FAD
:1046B000AFEAB5E002C0819311968C918823D9F7B7
:1046C0001F910F91FF90EF90DF90CF90BF90AF9030
:1046D0000895AF92BF92CF92DF92EF92FF920F9325
:1046E0001F938091FE01809381039091FF0190932D
:1046F000820180911802882309F44BC0892F90E031
:1047000020910E0130E0289FA001299F500D389F75
:10471000500D112420910F0130E0289FF001299FB6
:10472000F00D389FF00D112480917D0390917E0350
:104730008417950710F4642F07C0BF0162507040C2
:104740008617970708F4BC0100D000D070E080E025
:1047500090E09A0140E050E031977F0100E010E0E6
:10476000A7E0AA2EB12CC12CD12CEDB7FEB7A182A7
:10477000B282C382D482AA24BB2465010E9455332D
:1047800086E9861B8093AF050F900F900F900F90D6
:1047900003C087E98093AF0520917D0330917E03AC
:1047A00080918103482F50E02417350720F4809131
:1047B0005C01882341F580917A0290917B028070A0
:1047C000907C8050904CE1F4C90160EB75E044E0CE
:1047D00023E00E94F60489EA8093B4051092B5059F
:1047E000E0917A02F0917B02F170E253FC4FAFEA64
:1047F000B5E002C0819311968C918823D9F703C04C
:104800004217530708F71F910F91FF90EF90DF9029
:10481000CF90BF90AF9008952091600230916102D7
:10482000C9018070907C8050904CE1F48091270207
:104830008823C1F08091A5069091A606880F991F44
:10484000880F991F317083509D4F6AE570E00E9478
:10485000C5386F5A7E4FC90181539C4F49E050E0E3
:104860000E94350308951F920F920FB60F921124E4
:104870001F932F933F934F935F936F937F938F93E8
:104880009F93AF93BF93EF93FF9316B178940E94D9
:10489000D4318091A8069091A9069B01281B390B61
:1048A000C901895B9B4018F081E080933D017093C2
:1048B000A9066093A80613FD2AC08091AA069091CC
:1048C000AB06681B790BCB018F5E92408B5D9540E8
:1048D000A0F480918301882361F0E0913D01E930EB
:1048E00060F4F0E0EE0FFF1FE55EFE4F7183608322
:1048F00004C070937C0360937B0380913D018F5FC4
:1049000080933D01709385016093840104C070938E
:10491000AB066093AA06FF91EF91BF91AF919F9173
:104920008F917F916F915F914F913F912F911F9147
:104930000F900FBE0F901F901895AF92BF92CF921D
:10494000DF92EF92FF920F931F93CF93DF93CEEB03
:10495000D2E000E010E0F02EE12EF801EA5EFE4F1A
:1049600080810E942433BC01002349F4809101021C
:10497000882399F180911903682F70E02EC024E0FC
:10498000021759F58091FC018823F9F060917B03AF
:1049900070917C037595679561157105B1F420914F
:1049A000AC0684E0912FFC0143E0EE0FFF1F4A9517
:1049B000E1F7880F991FE80FF91FE20FF11DEE0FC5
:1049C000FF1FE255FD4F608171818091FB018823BB
:1049D00021F060914003709141034091AC0650E09A
:1049E0008F2D9E2DFC01B3E0EE0FFF1FBA95E1F76E
:1049F000880F991FE80FF91FE40FF51FEE0FFF1F37
:104A0000E255FD4F8881998120813181821B930B72
:104A1000998388838F2D9E2DFC0123E0EE0FFF1FCD
:104A20002A95E1F7880F991FE80FF91FE40FF51F8A
:104A3000EE0FFF1FE255FD4F20813181260F371FFA
:104A4000369527958F2D9E2DFC0173E0EE0FFF1FED
:104A50007A95E1F7880F991FE80FF91FE40FF51F0A
:104A6000EE0FFF1FE255FD4F31832083888199812E
:104A7000820F931F998388830F5F1F4F64960530C1
:104A8000110509F068CF80910102882309F043C025
:104A90008091BE029091BF0220911B02BC0180E078
:104AA00090E02223C1F40E94DE367B018C016091EC
:104AB000000270E0882777FD8095982F0E94E036ED
:104AC0009B01AC01C801B7010E94D63727E137EB43
:104AD00041ED58E317C00E94DE367B018C016091E6
:104AE000000270E0882777FD8095982F0E94E036BD
:104AF0009B01AC01C801B7010E94D6372FE632E115
:104B000043E05AE30E94D6370E94B23670937E0388
:104B100060937D030DC08091BE029091BF0203E0BF
:104B2000959587950A95E1F790937E0380937D0391
:104B30008091F801809382038091D2029091D302F8
:104B400020911B02BC0180E090E02223C1F40E946E
:104B5000DE367B018C016091080270E0882777FDCA
:104B60008095982F0E94E0369B01AC01C801B701E7
:104B70000E94D63727E137EB41ED58E317C00E947A
:104B8000DE367B018C016091080270E0882777FD9A
:104B90008095982F0E94E0369B01AC01C801B701B7
:104BA0000E94D6372FE632E143E05AE30E94D6371F
:104BB0000E94B2367093800360937F03809103025A
:104BC000882309F0E3C080910502882309F05FC0C3
:104BD0006091E6027091E70213E0759567951A956A
:104BE000E1F7882777FD8095982F0E94E036609343
:104BF0006F0370937003809371039093720300D0DE
:104C000000D0CDB6DEB60894C11CD11C0E94AD36D2
:104C1000209144023091450240E050E0E09046028D
:104C2000F090470200E010E0F601E082F18202839A
:104C30001383E12CB4E0FB2E012D112DAA24BB24FB
:104C400065010E9455330E94E03660936F037093B4
:104C5000700380937103909372030F900F900F90E5
:104C60000F9020E030E040E050E00E943E36882384
:104C70000CF0A7C080E090E0A0E0B0E080936F036C
:104C800090937003A0937103B09372039AC08091C4
:104C900023019091240160911201709113018617F4
:104CA000970740F0609114017091150186179707DE
:104CB00008F4BC0180E090E0685E73408040904062
:104CC000623FF3E07F07F0E08F07F0E09F0730F0EE
:104CD000A4E6AA2EB12CC12CD12C0AC02AE030E0C7
:104CE00040E050E00E94D838C901DA015C016D0152
:104CF000C601B5010E94DE367B018C01C601B501FB
:104D0000A60195010E9485380E94DE362AE037ED23
:104D100043EA5CE30E94D6379B01AC01C801B701AE
:104D20000E94DA357B018C01609146027091470246
:104D300080E090E00E94DE369B01AC01C801B70123
:104D40000E94D6372AE037ED43E25CE30E94D63773
:104D50007B018C0180911C03882379F060914402CF
:104D60007091450280E090E00E94DE369B01AC012C
:104D7000C801B7010E94DA351CC0609144027091ED
:104D8000450280E090E00E94DE3613C080917703F8
:104D90009091780397FF02C0059701C005966AE0DD
:104DA00070E00E94C538882777FD8095982F0E9473
:104DB000E03660936F037093700380937103909358
:104DC00072038091FA01882309F456C020910E03E2
:104DD00030910F03F3E035952795FA95E1F730937D
:104DE0007A032093790380918801882389F0809148
:104DF00060018F3029F430934B0220934A0208C09F
:104E0000813031F4309349022093480210926001BE
:104E100000D000D0B901882777FD8095982F209188
:104E200048023091490240E050E0E0904A02F090A0
:104E30004B0200E010E0E4E6AE2EB12CC12CD12CE8
:104E4000EDB7FEB7A182B282C382D482AA24BB246A
:104E500065010E9455330F900F900F900F906536AB
:104E6000710514F064E670E077FF02C060E070E066
:104E700070937A03609379038091AC068F5F80937F
:104E8000AC06883010F01092AC06DF91CF911F91E4
:104E90000F91FF90EF90DF90CF90BF90AF9008956B
:104EA000BF92CF92DF92EF92FF920F931F93DF9307
:104EB000CF93CDB7DEB764970FB6F894DEBF0FBEC1
:104EC000CDBF80910C01E82FFF27E7FDF095EE0F95
:104ED000FF1FE856FF4F85919491A2EFB3E001C008
:104EE0002D93FC01019624912223D1F7AAE3B5E08A
:104EF0008AEA90E001C02D93FC01019624912223BF
:104F0000D1F780911D038823B1F4A0E4B5E08FEAC6
:104F100090E001C02D93FC01019624912223D1F74A
:104F2000AAE4B5E089EB90E001C02D93FC01019665
:104F300024912223D1F780910C01882309F090C09D
:104F400080918D0390918E039C838B838091870346
:104F5000909188039E838D83809185039091860331
:104F600098878F8380918303909184039A878987A0
:104F7000609173037091740380917503909176032F
:104F800020E030E044EB53E40E9445360E94AD3609
:104F90007C876B8780918B0390918C036AE070E033
:104FA0000E94B1387E876D876E010894C11CD11CA8
:104FB000EE24FF240DE510E0F701EE0FFF1FE05493
:104FC000FF4F85919491D801A153BC4F01C02D93FF
:104FD000FC01019624912223D1F7F6018081918171
:104FE0006FEA75E04AE050E00E943E03D801A0520B
:104FF000BC4FFC0102C08D93319680818823D9F784
:105000000894E11CF11C025E1F4F82E090E0C80E84
:10501000D91E97E0E916F10479F660919103709139
:10502000920380E090E04FEA55E021E00E94C30542
:10503000ACE3B4E0EFEAF5E002C08D9331968081F5
:105040008823D9F780914203882351F0E3E4F3E009
:10505000ACE1B5E002C08D93319680818823D9F709
:1050600080910C01813009F093C080E090E02DE543
:1050700030E0FC0143E0EE0FFF1F4A95E1F7D90154
:10508000A153BC4FE956FC4F02C04D93319640816D
:105090004423D9F70196225E3F4F8730910549F7A7
:1050A000FF243EE1B32EE5E0FE1619F427E0F22ED0
:1050B00005C0F6E0FF1510F0EF2C03C09EEFE92EBF
:1050C000EF0C0F2D10E0F801E752FA4F808190E0CD
:1050D0006FEA75E04AE050E00E943E03EB9C6001FD
:1050E0001124D601AC5CBB4FFC0102C08D933196FC
:1050F00080818823D9F7F801ED51FA4F808190E043
:105100006FEA75E04AE050E00E943E03D601A65CDB
:10511000BB4FFC0102C08D93319680818823D9F763
:1051200003511A4FF801808190E06FEA75E04AE080
:1051300050E00E943E03D601A05CBB4FFC0102C0C0
:105140008D93319680818823D9F7F394F8E0FF1589
:1051500008F0A9CFA6E1B4E0E0E0F1E002C08D9351
:10516000319680818823D9F7ACE1B4E0E2E0F1E048
:1051700002C08D93319680818823D9F7A2E2B4E0F2
:10518000E4E0F1E002C08D93319680818823D9F765
:1051900080910C01823009F055C08091F705898318
:1051A0001A828091F8058B831C828091F9058D838A
:1051B0001E828091FA058F8318868091FB0589876E
:1051C0001A868091FC058B871C868091FD058D8752
:1051D0001E866E010894C11CD11CEE24FF240DE52F
:1051E00010E0F701EE0FFF1FE253FF4F85919491FE
:1051F000D801A153BC4F01C02D93FC01019624910D
:105200002223D1F7F601808191816FEA75E04AE0AF
:1052100050E00E943E03D801AD51BC4FFC0102C0DA
:105220008D93319680818823D9F70894E11CF11C75
:10523000025E1F4F82E090E0C80ED91E97E0E9168B
:10524000F10479F680910C01833009F0E9C00E94E5
:105250009D2487E98093AF0580917D0390917E0323
:1052600060EB75E044E023E00E94F60489EA809355
:10527000B4051092B505A3E0B4E0EFEAF5E002C092
:105280008D93319680818823D9F78FEB8093AF057A
:1052900080917F039091800360EB75E044E023E010
:1052A0000E94F60489EA8093B4051092B505ABEF2D
:1052B000B3E0EFEAF5E002C08D9331968081882358
:1052C000D9F720E030E04DE550E0F901EE0FFF1F87
:1052D000E452FF4F85919491DA01A153BC4F01C074
:1052E0006D93FC01019664916623D1F72F5F3F4FC8
:1052F000425E5F4F2730310541F78091070290E011
:105300006FEA75E04AE050E00E943E03FC01AAE922
:10531000B4E002C08D93319680818823D9F78091C3
:10532000FD01E82FF0E0EE0FFF1FEC56FF4F8591D7
:105330009491A0E4B4E001C02D93FC010196249166
:105340002223D1F78091000290E06FEA75E04AE0F5
:1053500050E00E943E03FC01AEE5B4E002C08D9334
:10536000319680818823D9F78091FE0190E06FEA21
:1053700075E04AE050E00E943E03FC01ACE7B4E077
:1053800002C08D93319680818823D9F780910702DE
:10539000E82FF0E0EE0FFF1FEC56FF4F8591949140
:1053A000AAE9B4E001C02D93FC01019624912223C7
:1053B000D1F78091080290E06FEA75E04AE050E092
:1053C0000E943E03FC01A8EBB4E002C08D9331962D
:1053D00080818823D9F78091FF0190E06FEA75E022
:1053E0004AE050E00E943E03FC01A6EDB4E002C09A
:1053F0008D93319680818823D9F780910102E82F1F
:10540000F0E0EE0FFF1FEC56FF4F85919491A4EF53
:10541000B4E001C02D93FC01019624912223D1F721
:1054200080910C01843009F0BDC080917903909186
:105430007A036FEA75E04AE050E00E943E03E0E044
:10544000AE2FB0E0A155BA4F8C91EF5F8823C1F722
:1054500085E28C93F0E0E155FA4F1082A4E0B4E0CD
:10546000EFEAF5E002C08D93319680818823D9F769
:1054700020E030E04DE550E0F901EE0FFF1FE6516E
:10548000FF4F85919491DA01A153BC4F01C06D93F8
:10549000FC01019664916623D1F72F5F3F4F425E76
:1054A0005F4F2630310541F78091FA01E82FF0E097
:1054B000EE0FFF1FEC56FF4F85919491A0E4B4E0EE
:1054C00001C02D93FC01019624912223D1F78091F4
:1054D0006001882329F4AEE5B4E0E6E0F1E013C012
:1054E00090E06FEA75E04AE050E00E943E03FC0164
:1054F000AEE5B4E002C08D93319680818823D9F760
:1055000005C08D93319680818823D9F78091FB0166
:10551000E82FF0E0EE0FFF1FEC56FF4F85919491BE
:10552000ACE7B4E001C02D93FC0101962491222345
:10553000D1F78091FC01E82FF0E0EE0FFF1FEC5651
:10554000FF4F85919491AAE9B4E001C02D93FC012D
:10555000019624912223D1F780914A0290914B0227
:105560006FEA75E04AE050E00E943E03FC01A8EBC0
:10557000B4E002C08D93319680818823D9F7809161
:105580004802909149026FEA75E04AE050E00E94BB
:105590003E03FC01A6EDB4E002C08D9331968081FC
:1055A0008823D9F780910C01853009F09CC0609167
:1055B0006F037091700380917103909172030E9448
:1055C000AD36DC01CB016FEA75E044E023E00E94D8
:1055D000F6048AE98093B3051092B405A3E0B4E021
:1055E000EFEAF5E002C08D93319680818823D9F7E8
:1055F00020E030E04DE550E0F901EE0FFF1FEA50EA
:10560000FF4F85919491DA01A153BC4F01C06D9376
:10561000FC01019664916623D1F72F5F3F4F425EF4
:105620005F4F2530310541F780910202E82FF0E00D
:10563000EE0FFF1FEC56FF4F85919491A0E4B4E06C
:1056400001C02D93FC01019624912223D1F7809172
:105650000402E82FF0E0EE0FFF1FEC56FF4F85919C
:105660009491AEE5B4E001C02D93FC010196249124
:105670002223D1F780910502E82FF0E0EE0FFF1F03
:10568000EC56FF4F85919491ACE7B4E001C02D93A7
:10569000FC01019624912223D1F78091460290913A
:1056A00047026FEA75E04AE050E00E943E03FC01C9
:1056B000AAE9B4E002C08D93319680818823D9F79E
:1056C00080914402909145026FEA75E04AE050E013
:1056D0000E943E03FC01A8EBB4E002C08D9331961A
:1056E00080818823D9F780910C01863009F0B3C0FE
:1056F00020E030E04DE550E0F901EE0FFF1FE050F3
:10570000FF4F85919491DA01A153BC4F01C06D9375
:10571000FC01019664916623D1F72F5F3F4F425EF3
:105720005F4F2830310541F780911602E82FF0E0F5
:10573000EE0FFF1FEC56FF4F85919491A0E4B4E06B
:1057400001C02D93FC01019624912223D1F7809171
:105750001702E82FF0E0EE0FFF1FEC56FF4F859188
:105760009491AEE5B4E001C02D93FC010196249123
:105770002223D1F780912302E82FF0E0EE0FFF1FE4
:10578000EC56FF4F85919491ACE7B4E001C02D93A6
:10579000FC01019624912223D1F780911502E82F74
:1057A000F0E0EE0FFF1FEC56FF4F85919491AAE9B0
:1057B000B4E001C02D93FC01019624912223D1F77E
:1057C00080910D02E82FF0E0EE0FFF1FEC56FF4F27
:1057D00085919491A8EBB4E001C02D93FC01019652
:1057E00024912223D1F780912A02E82FF0E0EE0FD6
:1057F000FF1FEC56FF4F85919491A6EDB4E001C0D8
:105800002D93FC01019624912223D1F7809124024B
:10581000E82FF0E0EE0FFF1FEC56FF4F85919491BB
:10582000A4EFB4E001C02D93FC0101962491222342
:10583000D1F780911A0290E06FEA75E04AE050E0FB
:105840000E943E03FC01A2E1B5E002C08D933196B7
:1058500080818823D9F780910C01873009F096C0A8
:1058600020E030E04DE550E0F901EE0FFF1FE05F72
:10587000FE4F85919491DA01A153BC4F01C06D9305
:10588000FC01019664916623D1F72F5F3F4F425E82
:105890005F4F2530310541F780911302882329F0AD
:1058A000A0E4B4E08EE191E00DC0A0E4B4E08AE1B0
:1058B00091E001C02D93FC01019624912223D1F7A0
:1058C00006C02D93FC01019624912223D1F78091EB
:1058D0001B02882329F4AEE5B4E085E291E00DC017
:1058E000AEE5B4E082E291E001C02D93FC010196A7
:1058F00024912223D1F706C02D93FC010196249117
:105900002223D1F780912202E82FF0E0EE0FFF1F53
:10591000EC56FF4F85919491ACE7B4E001C02D9314
:10592000FC01019624912223D1F780916101882303
:1059300029F4AAE9B4E0E6E0F1E013C090E06FEAF0
:1059400075E04AE050E00E943E03FC01AAE9B4E0A1
:1059500002C08D93319680818823D9F705C08D933D
:10596000319680818823D9F78091300290E06FEAE8
:1059700075E04AE050E00E943E03FC01A8EBB4E071
:1059800002C08D93319680818823D9F780910C01D4
:10599000883009F067C08091340289831A8280912F
:1059A00035028B831C82809136028D831E8280910A
:1059B00037028F83188680910A0289871A86809120
:1059C0000B028B871C866E010894C11CD11C00E061
:1059D00010E0EDE5EE2EF12CF801EE0FFF1FE65D75
:1059E000FE4F85919491D701A153BC4F01C02D93D7
:1059F000FC01019624912223D1F7063099F0F6019B
:105A0000808191816FEA75E04AE050E00E943E0398
:105A1000D701AD51BC4FFC0102C08D9331968081FE
:105A20008823D9F70F5F1F4F8EE190E0E80EF91E33
:105A3000E2E0F0E0CE0EDF1E0730110569F680913E
:105A40000602E82FF0E0EE0FFF1FEC56FF4F8591A6
:105A50009491A4EFB4E001C02D93FC010196249130
:105A60002223D1F780910C01893014F010920C019F
:105A70000E94CA0A64960FB6F894DEBF0FBECDBF6F
:105A8000CF91DF911F910F91FF90EF90DF90CF901A
:105A9000BF900895EF92FF920F931F93109293037C
:105AA00080916C0190916D01019690936D018093AE
:105AB0006C0180917801882311F00C940000E09132
:105AC0003002E09309011092860180912F02882311
:105AD00089F0F0E0EE0FFF1FE55EFE4F0190F081D0
:105AE000E02D26E0E134F207E8F4E957F540E8F06C
:105AF00082E019C08091E6019091E701A091E80150
:105B0000B091E901209114033091150340911603DF
:105B10005091170382239323A423B5230097A10553
:105B2000B10519F081E08093860190918601809102
:105B30008701981711F00E94060C809186018093CE
:105B4000870180915A01863018F087E061E002C039
:105B500087E060E00E94CD320E94C6317B018C015B
:105B60002091CB053091CC054091CD055091CE05CB
:105B7000DC01CB01821B930BA40BB50B8436910582
:105B8000A105B10508F446C02C593F4F4F4F5F4F58
:105B90002093CB053093CC054093CD055093CE0593
:105BA00080915A018F5F80935A0180915B018F5FD2
:105BB00080935B0190E080915D01882309F491E07E
:105BC00090935D010E943904809104028823D1F0F2
:105BD00060917303709174038091750390917603C3
:105BE00020916F03309170034091710350917203C3
:105BF0000E94DA3560937303709374038093750386
:105C00009093760380918901882321F48CE660E0EB
:105C10000E9469118091CF059091D005A091D10586
:105C2000B091D205E81AF90A0A0B1B0B22E3E2161F
:105C3000F1040105110508F433C2C296A11DB11D7E
:105C40008093CF059093D005A093D105B093D20552
:105C50008091C7059091C805A091C905B091CA056A
:105C60000097A105B10581F48091C3059091C40509
:105C7000A091C505B091C6058093C7059093C8054E
:105C8000A093C905B093CA052091C7053091C805F6
:105C90004091C9055091CA05EE24FF248701E21AFC
:105CA000F30A040B150BE222F32204231523D80177
:105CB000C70180959095A095B09582239323A42346
:105CC000B5238093C7059093C805A093C905B093E9
:105CD000CA0580E0E81682E0F80680E0080780E068
:105CE000180709F4B6C021E0E21622E0F20620E02F
:105CF000020720E01207E0F580E1E816F104010553
:105D0000110509F4A0C021E1E216F1040105110515
:105D1000B0F482E0E816F1040105110509F48BC026
:105D200028E0E216F1040105110509F486C081E0BE
:105D3000E816F1040105110509F079C07AC020E8E0
:105D4000E216F1040105110509F479C080E0E816B6
:105D500081E0F80680E0080780E0180709F475C0C4
:105D600020E2E216F1040105110509F060C069C0E6
:105D700080E0E81680E0F80681E0080780E0180778
:105D800009F465C021E0E21620E0F20621E00207F6
:105D900020E01207F0F480E0E81688E0F80680E0E2
:105DA000080780E0180709F45EC020E0E21620E151
:105DB000F20620E0020720E0120709F456C080E056
:105DC000E81684E0F80680E0080780E0180779F517
:105DD00044C020E0E21620E0F20624E0020720E0C2
:105DE0001207C9F181E0E81680E0F80684E00807B0
:105DF00080E0180750F420E0E21620E0F20622E0EE
:105E0000020720E0120799F432C080E0E81680E033
:105E1000F80688E0080780E0180719F120E0E2168C
:105E200020E0F20620E2020720E01207C1F090E035
:105E30001FC094E61DC095E61BC099E619C09AE6FE
:105E400017C09BE615C09DE613C09EE611C092E701
:105E50000FC09FE60DC09BE30BC090E709C095E71C
:105E600007C099E405C097E703C09CED01C092EF1D
:105E700080918901882331F4892F60E00E946911A3
:105E80000E94811C0E949D2480917B0190917C0145
:105E9000089760F40E94F60980916B0390916C035F
:105EA000CC9790935F0180935E01FAC080911C03B0
:105EB000882349F081E080931D038091880181301F
:105EC00011F40E94D20B80911D03882341F0809130
:105ED0001C03882321F410921D03109288018091E5
:105EE0008801882319F00E945027DAC00E94980385
:105EF0008091120380FF0AC06091AC027091AD02E4
:105F00008091AA029091AB020E94ED0D8091FD015B
:105F1000882311F00E94692380910702882311F0E1
:105F20000E9445088091FA01882381F08091F9014F
:105F300090E02091790330917A038217930724F03F
:105F400080915C01882311F00E94821F80910202DF
:105F5000882339F160916F03709170038091710310
:105F60009091720320E030E040E251E40E94453617
:105F70007B018C0160910B0270E0882777FD809592
:105F8000982F0E94E0369B01AC01C801B7010E9426
:105F90003E3687FD04C080915C01882311F00E9489
:105FA000D90880910402882351F00E946F0388234E
:105FB00021F080915C01882311F00E94B71F0E949C
:105FC0007B080E942B090E94240D809115028823D2
:105FD00011F00E94C32240916B0350916C032091F9
:105FE0005E0130915F01C901CC968417950770F569
:105FF000205C3F4F2417350720F450935F014093F6
:106000005E0180911E02882309F140919E02509109
:106010009F0220E030E0F901E155FA4FD901A85C78
:10602000BD4F8C9180832F5F3F4F2A30310599F708
:106030001092B905DA01B170A153BC4FEFEAF5E057
:1060400002C08D93319680818823D9F78091120305
:1060500082FF04C00E940C240E94B40980911203A4
:1060600081FF04C00E94761D0E944122809112038C
:1060700083FF12C080910C02882371F00E94531F8D
:106080000E947F0A0E940E1D0E944F0A0E94E11E7C
:106090000E944A1E0E94EB1F0E9489060E947F0BED
:1060A00080915B01853050F010925B0190E080910F
:1060B0005C01882309F491E090935C010E94C63151
:1060C000209166013091670140916801509169010A
:1060D00028513C4F4F4F5F4F261737074807590746
:1060E00008F096C0209366013093670140936801E1
:1060F0005093690110925A0180916C0190916D0149
:106100009093CC018093CB0110926D0110926C01A1
:1061100080916E0190916F019093CE018093CD019B
:1061200010926F0110926E01809170019091710137
:106130009093D0018093CF01109271011092700161
:1061400080916B0390916C03019690936C03809304
:106150006B0380918901882311F40E94BC0C80910B
:106160006B01882319F410923D0303C08150809382
:106170006B0180916A01882319F0815080936A0134
:1061800080911C03882349F48091A5069091A6066E
:1061900090931F0380931E0316C080916D0390910E
:1061A0006E03019690936E0380936D03809191032B
:1061B0009091920301969093920380939103109291
:1061C00088010E94980380917B0190917C01019647
:1061D00090937C0180937B0180916101813051F427
:1061E00080918801882331F08EEC60E00E94691173
:1061F0001092610180916101882319F08150809390
:10620000610180916001882319F0815080936001C1
:1062100081E00E94B31B61E070E080E090E00E94AA
:10622000FA311F910F91FF90EF90089583E497E06A
:1062300040E052EC61E070E00E9428348091C000A0
:1062400082608093C0001092C50080E18093C400FA
:1062500083E497E00E94093584B18C6284B9249864
:10626000569A529884E160E00E948E3281E160E0AB
:106270000E948E3281E160E00E948E3287E061E010
:106280000E948E323B98F89480916C0083FD0AC086
:106290008091680082608093680080916C008860C3
:1062A00080936C0078940E9482100E94E20C64EF4C
:1062B00071E080E090E00E94FA3180911B02882317
:1062C00011F081E001C083E00E9421330E94540C50
:1062D0000E9498030895F999FECF72BD61BDF89AA6
:1062E00080B50895F999FECF1FBA72BD61BD40BD5A
:1062F0000FB6F894FA9AF99A0FBE08951F920F926A
:106300000FB60F9211242F933F938F939F93AF93C8
:10631000BF938091B6069091B706A091B806B09150
:10632000B9063091BA060196A11DB11D232F2D5F2C
:106330002D3720F02D570196A11DB11D2093BA06CF
:106340008093B6069093B706A093B806B093B906AB
:106350008091B2069091B306A091B406B091B506B3
:106360000196A11DB11D8093B2069093B306A09330
:10637000B406B093B506BF91AF919F918F913F91B5
:106380002F910F900FBE0F901F9018958FB7F89414
:106390002091B6063091B7064091B8065091B906E3
:1063A0008FBFB901CA0108959FB7F8942091B20632
:1063B0003091B3064091B4065091B50686B5A89BBE
:1063C00006C08F3F21F02F5F3F4F4F4F5F4F9FBF62
:1063D000542F432F322F2227280F311D411D511DCD
:1063E00082E0220F331F441F551F8A95D1F7B90150
:1063F000CA0108959B01AC017FB7F8948091B20661
:106400009091B306A091B406B091B50666B5A89B6D
:1064100005C06F3F19F00196A11DB11D7FBFBA2FB6
:10642000A92F982F8827860F911DA11DB11D62E00D
:10643000880F991FAA1FBB1F6A95D1F7BC012DC0F9
:10644000FFB7F8948091B2069091B306A091B4067C
:10645000B091B506E6B5A89B05C0EF3F19F00196CF
:10646000A11DB11DFFBFBA2FA92F982F88278E0F0E
:10647000911DA11DB11DE2E0880F991FAA1FBB1F2E
:10648000EA95D1F7861B970B885E9340C8F221509E
:1064900030404040504068517C4F21153105410546
:1064A000510571F60895789484B5826084BD84B5F1
:1064B000816084BD85B5826085BD85B5816085BDFF
:1064C000EEE6F0E0808181608083E1E8F0E0108218
:1064D000808182608083808181608083E0E8F0E059
:1064E000808181608083E1EBF0E080818460808343
:1064F000E0EBF0E0808181608083EAE7F0E080817A
:1065000084608083808182608083808181608083D9
:106510008081806880831092C1000895CF93DF93BB
:10652000482F50E0CA0188529A4FFC0134914C53D5
:106530005A4FFA018491882369F190E0880F991FDE
:10654000FC01EA55FA4FA591B491FC01E055FA4FD0
:10655000C591D491662351F42FB7F8948C91932F61
:10656000909589238C93888189230BC0623061F4D4
:106570002FB7F8948C91932F909589238C938881D1
:10658000832B88832FBF06C09FB7F8948C91832BF1
:106590008C939FBFDF91CF910895482F50E0CA019F
:1065A00084519A4FFC012491CA0188529A4FFC01F0
:1065B00094914C535A4FFA013491332309F440C05B
:1065C000222351F1233071F0243028F42130A1F03E
:1065D000223011F514C02630B1F02730C1F024303C
:1065E000D9F404C0809180008F7703C0809180002F
:1065F0008F7D8093800010C084B58F7702C084B5F2
:106600008F7D84BD09C08091B0008F7703C08091D9
:10661000B0008F7D8093B000E32FF0E0EE0FFF1FFE
:10662000E055FA4FA591B4912FB7F894662321F461
:106630008C919095892302C08C91892B8C932FBFCC
:10664000089580933E010895982F8E3008F09E5053
:10665000977080913E018295880F880F807C892BEE
:1066600080937C0080917A00806480937A0080918E
:106670007A0086FDFCCF2091780040917900942F1C
:1066800080E030E0282B392BC9010895CF93DF93A8
:106690000E9453320E941631CAEDD3E30E944A2D64
:1066A0002097E1F30E94DA33F9CF2F923F924F9275
:1066B0005F926F927F928F929F92AF92BF92CF9292
:1066C000DF92EF92FF920F931F93DF93CF93CDB79B
:1066D000DEB73B014C0119012A016D897E898F8942
:1066E000988D6A197B098C099D09621A730A840ABC
:1066F000950AA40193010E948538E218F308040961
:106700001509A80197010E94FA382A0D3B1D4C1D5E
:106710005D1DB901CA01CF91DF911F910F91FF90CB
:10672000EF90DF90CF90BF90AF909F908F907F9031
:106730006F905F904F903F902F90089508951F9213
:106740000F920FB60F9211242F933F934F938F9375
:106750009F93EF93FF938091C00082FD1DC04091F5
:10676000C6002091FB063091FC062F5F3F4F2F7330
:1067700030708091FD069091FE062817390771F060
:10678000E091FB06F091FC06E554F94F408330930D
:10679000FC062093FB0602C08091C600FF91EF919A
:1067A0009F918F914F913F912F910F900FBE0F901E
:1067B0001F901895E0914F07F0915007E05CFF4F54
:1067C0008191919120813181821B930B8F73907005
:1067D000892B11F00E949E3308951F920F920FB6DD
:1067E0000F9211242F933F938F939F93EF93FF93D7
:1067F00020913F07309140078091410790914207D7
:106800002817390731F48091C1008F7D8093C10032
:1068100014C0E0914107F0914207E150F94F208107
:10682000809141079091420701968F7390709093E9
:106830004207809341072093C600FF91EF919F91FB
:106840008F913F912F910F900FBE0F901F90189531
:10685000AF92BF92DF92EF92FF920F931F93CF936D
:10686000DF93EC017A018B01DD24403081EE580783
:1068700080E0680780E0780711F0DD24D39491E090
:10688000A92EB12CEC89FD89DD2069F0C50108A095
:1068900002C0880F991F0A94E2F7808360E079E0D4
:1068A0008DE390E005C0108260E874E88EE190E02E
:1068B000A80197010E94D8382150304040405040F4
:1068C000569547953795279580E12030380720F079
:1068D000DD2011F0DD24D6CFE889F9893083EA89FB
:1068E000FB89208319A2EE89FF89408121E030E0F5
:1068F000C9010C8C02C0880F991F0A94E2F7482B3B
:106900004083EE89FF894081C9010D8C02C0880F48
:10691000991F0A94E2F7482B4083EE89FF89408152
:10692000C9010E8C02C0880F991F0A94E2F7482B08
:106930004083EE89FF8980810F8C02C0220F331FB4
:106940000A94E2F7209528232083DF91CF911F91AD
:106950000F91FF90EF90DF90BF90AF900895DC0112
:106960001C96ED91FC911D97E05CFF4F21913191B8
:1069700080819181281B390B2F733070C9010895D4
:10698000DC011C96ED91FC911D97E05CFF4F20818E
:106990003181E054F040DF01AE5BBF4F8D919C919F
:1069A00011972817390719F42FEF3FEF07C08D9182
:1069B0009C91E80FF91F8081282F30E0C9010895CC
:1069C000DC011C96ED91FC911D97E05CFF4F20814E
:1069D0003181E054F040DF01AE5BBF4F8D919C915F
:1069E00011972817390719F42FEF3FEF10C08D9139
:1069F0009C911197E80FF91F20818D919C9111971F
:106A000001968F73907011969C938E9330E0C9011C
:106A10000895DC0191968C919197882339F05496D2
:106A2000ED91FC915597808186FFF9CF91961C924C
:106A30000895CF93DF93EC01EE85FF85E05CFF4F77
:106A400020813181E054F0402F5F3F4F2F73307031
:106A5000DF01AE5BBF4F8D919C91119728173907CD
:106A6000D1F3E05CFF4F80819181E054F040E80F6A
:106A7000F91F6083EE85FF85E05CFF4F3183208343
:106A8000EE89FF89208181E090E00F8C02C0880FA1
:106A9000991F0A94E2F7282B208381E089A3EC89CF
:106AA000FD8980818064808381E090E0DF91CF91D7
:106AB0000895109246071092450788EE93E0A0E0F3
:106AC000B0E08093470790934807A0934907B0939D
:106AD0004A078DE491E090934407809343078BEB42
:106AE00096E09093500780934F078FEF96E0909336
:106AF00052078093510785EC90E090935407809360
:106B0000530784EC90E0909356078093550780ECF0
:106B100090E0909358078093570781EC90E0909312
:106B20005A078093590782EC90E090935C0780931A
:106B30005B0786EC90E090935E0780935D0784E0AE
:106B400080935F0783E08093600787E0809361070D
:106B500085E08093620781E0809363070895CF9278
:106B6000DF92EF92FF920F931F93CF93DF937C01FD
:106B70006B018A01C0E0D0E00FC0D6016D916D01BC
:106B8000D701ED91FC910190F081E02DC7010995AD
:106B9000C80FD91F015010400115110571F7CE0122
:106BA000DF91CF911F910F91FF90EF90DF90CF90E9
:106BB00008955058BB27AA270ED0A9C169D130F03B
:106BC0006ED120F031F49F3F11F41EF45EC10EF43B
:106BD000E095E7FB54C1E92FBCD180F3BA176207F7
:106BE00073078407950718F071F49EF5D4C10EF46D
:106BF000E0950B2EBA2FA02D0B01B90190010C01CD
:106C0000CA01A0011124FF27591B99F0593F50F4E4
:106C1000503E68F11A16F040A22F232F342F44273C
:106C2000585FF3CF469537952795A795F040539534
:106C3000C9F77EF41F16BA0B620B730B840BBAF004
:106C40009150A1F0FF0FBB1F661F771F881FC2F76F
:106C50000EC0BA0F621F731F841F48F48795779583
:106C60006795B795F7959E3F08F0B3CF9395880F3A
:106C700008F09927EE0F979587950895DCD008F4D2
:106C800081E0089514D1E39553C10CD040C107D1E0
:106C900040F0FED030F021F45F3F19F0F0C0511108
:106CA0007BC1F3C056D198F39923C9F35523B1F3AF
:106CB000951B550BBB27AA2762177307840738F06B
:106CC0009F5F5F4F220F331F441FAA1FA9F333D0CA
:106CD0000E2E3AF0E0E830D091505040E695001C7E
:106CE000CAF729D0FE2F27D0660F771F881FBB1F3A
:106CF000261737074807AB07B0E809F0BB0B802D14
:106D0000BF01FF2793585F4F2AF09E3F510568F05F
:106D1000B6C042C15F3FECF3983EDCF386957795B1
:106D20006795B795F7959F5FC9F7880F911D969561
:106D3000879597F90895E1E0660F771F881FBB1FBD
:106D4000621773078407BA0720F0621B730B840B6A
:106D5000BA0BEE1F88F7E095089504D06894B1113E
:106D60001BC10895FED088F09F5790F0B92F992746
:106D7000B751A0F0D1F0660F771F881F991F1AF046
:106D8000BA95C9F712C0B13081F005D1B1E00895CC
:106D900002C1672F782F8827B85F39F0B93FCCF34D
:106DA000869577956795B395D9F73EF4909580953C
:106DB000709561957F4F8F4F9F4F0895E89409C05C
:106DC00097FB3EF490958095709561957F4F8F4F1E
:106DD0009F4F9923A9F0F92F96E9BB279395F69534
:106DE000879577956795B795F111F8CFFAF4BB0FB2
:106DF00011F460FF1BC06F5F7F4F8F4F9F4F16C016
:106E0000882311F096E911C0772321F09EE8872F9F
:106E1000762F05C0662371F096E8862F70E060E05B
:106E20002AF09A95660F771F881FDAF7880F9695D4
:106E3000879597F90895990F0008550FAA0BE0E878
:106E4000FEEF16161706E807F907C0F0121613062C
:106E5000E407F50798F0621B730B840B950B39F46C
:106E60000A2661F0232B242B252B21F408950A26D2
:106E700009F4A140A6958FEF811D811D089597F912
:106E80009F6780E870E060E008959FEF80EC0895D0
:106E900000240A94161617061806090608950024F9
:106EA0000A9412161306140605060895EECF59D05B
:106EB000E8F3E894EFEFBB273FE048EC5FE76B3D7A
:106EC00073078407950708F1FF279F57B25A6A4D49
:106ED0007F40894CF04032F4BE556542704F864386
:106EE000FF4F0894EE1F915030F0BB0F661F771FC5
:106EF000881FFF1FEBCF9EE7882332F0BB0F661F72
:106F0000771F881F9A95C1F79395E095B8C0092E11
:106F10000394000C11F4882352F0BB0F40F4BF2BF4
:106F200011F460FF04C06F5F7F4F8F4F9F4F089534
:106F3000EF93E0FF06C0A2EA2AED3FE049EC5FEBE9
:106F40004ADEE5DF0F90039401FC9058E8E6F0E09C
:106F5000A6C057FD9058440F551F59F05F3F71F080
:106F60004795880F97FB991F61F09F3F79F08795B0
:106F70000895121613061406551FF2CF4695F1DF39
:106F800008C0161617061806991FF1CF86957105C9
:106F9000610508940895E894BB2766277727CB01FD
:106FA00097F9089548DF08F48FEF08950BD0AFCF1D
:106FB0006FDF28F074DF18F0952309F060CF65CFFC
:106FC0001124EACFC6DFA0F3959FD1F3950F50E0CF
:106FD000551F629FF001729FBB27F00DB11D639F8B
:106FE000AA27F00DB11DAA1F649F6627B00DA11D31
:106FF000661F829F2227B00DA11D621F739FB00DD7
:10700000A11D621F839FA00D611D221F749F332746
:10701000A00D611D231F849F600D211D822F762FDF
:107020006A2F11249F5750408AF0E1F088234AF0DC
:10703000EE0FFF1FBB1F661F771F881F9150504028
:10704000A9F79E3F510570F01ACFA6CF5F3FECF332
:10705000983EDCF3869577956795B795F795E79514
:107060009F5FC1F7FE2B880F911D9695879597F925
:1070700008959F931CDF0F9007FCEE5F59CF9F3F51
:1070800049F0915028F4869577956795B7959F5F5D
:1070900080389F4F880F9695879597F908959F930D
:1070A0008F937F936F93FF93EF939B01AC017EDFF0
:1070B000EF91FF9105D02F913F914F915F9176CF46
:1070C000DF93CF931F930F93FF92EF92DF927B0199
:1070D0008C01689405C0DA2EEF0174DFFE01E8949C
:1070E000A5912591359145915591AEF3EF0173DD51
:1070F000FE019701A801DA9479F7DF90EF90FF90F5
:107100000F911F91CF91DF910895629FD001739FDE
:10711000F001829FE00DF11D649FE00DF11D929F33
:10712000F00D839FF00D749FF00D659FF00D992772
:10713000729FB00DE11DF91F639FB00DE11DF91F96
:10714000BD01CF011124089587FB082E062687FD77
:10715000819567FD619569D00EF4919507FC819545
:107160000895AA1BBB1B51E107C0AA1FBB1FA6178E
:10717000B70710F0A61BB70B881F991F5A95A9F7E0
:1071800080959095BC01CD01089597FB092E0726A7
:107190000AD077FD04D0E5DF06D000201AF4709500
:1071A00061957F4F0895F6F7909581959F4F0895CB
:1071B000A1E21A2EAA1BBB1BFD010DC0AA1FBB1FFB
:1071C000EE1FFF1FA217B307E407F50720F0A21B6D
:1071D000B30BE40BF50B661F771F881F991F1A94DA
:1071E00069F760957095809590959B01AC01BD0104
:1071F000CF01089597FB092E05260ED057FD04D028
:10720000D7DF0AD0001C38F4509540953095219571
:107210003F4F4F4F5F4F0895F6F7909580957095CB
:1072200061957F4F8F4F9F4F0895991B79E004C060
:10723000991F961708F0961B881F7A95C9F78095B5
:107240000895EE0FFF1F0590F491E02D0994F89436
:02725000FFCF6E
:107252005000490044002D00FF080A030101222AC0
:1072620010104C046C070E100F1111DC05DC05DC4C
:1072720005DC05DC05DC05DC05DC05DC05DC05DC04
:1072820005DC05DC05DC05DC05DC0500000101A7E9
:10729200A8BBB97AA7DFBBA5A6000000001935AFCD
:0A72A20035AF34E034C03409350084
:00000001FF
